Archive member included because of file (symbol)

E:/Program Files/Rowley Associates Limited/CrossWorks for ARM 1.3/lib/libm_v4t_a_ni_le.a(sf-wrapper.o)
                              ARM Flash Debug/sfpdiag.o (__floatsisf)
E:/Program Files/Rowley Associates Limited/CrossWorks for ARM 1.3/lib/libm_v4t_a_ni_le.a(df-wrapper.o)
                              ARM Flash Debug/sfpdiag.o (__extendsfdf2)
E:/Program Files/Rowley Associates Limited/CrossWorks for ARM 1.3/lib/libc_v4t_a_ni_le.a(__int32_udivmod.o)
                              ARM Flash Debug/pll.o (__udivsi3)
E:/Program Files/Rowley Associates Limited/CrossWorks for ARM 1.3/lib/libc_v4t_a_ni_le.a(strlen.o)
                              ARM Flash Debug/nvstore.o (strlen)
E:/Program Files/Rowley Associates Limited/CrossWorks for ARM 1.3/lib/libc_v4t_a_ni_le.a(memcpy.o)
                              ARM Flash Debug/uip_arp.o (memcpy)
E:/Program Files/Rowley Associates Limited/CrossWorks for ARM 1.3/lib/libc_v4t_a_ni_le.a(memset.o)
                              ARM Flash Debug/uip_arp.o (memset)
E:/Program Files/Rowley Associates Limited/CrossWorks for ARM 1.3/lib/libc_v4t_a_ni_le.a(strncpy.o)
                              ARM Flash Debug/nvstore.o (strncpy)
E:/Program Files/Rowley Associates Limited/CrossWorks for ARM 1.3/lib/libc_v4t_a_ni_le.a(strtol.o)
                              ARM Flash Debug/ee24lc256.o (strtol)
E:/Program Files/Rowley Associates Limited/CrossWorks for ARM 1.3/lib/libc_v4t_a_ni_le.a(errno.o)
                              E:/Program Files/Rowley Associates Limited/CrossWorks for ARM 1.3/lib/libc_v4t_a_ni_le.a(strtol.o) (errno)
E:/Program Files/Rowley Associates Limited/CrossWorks for ARM 1.3/lib/libc_v4t_a_ni_le.a(printf.o)
                              ARM Flash Debug/clivar.o (printf)
E:/Program Files/Rowley Associates Limited/CrossWorks for ARM 1.3/lib/libc_v4t_a_ni_le.a(sprintf.o)
                              ARM Flash Debug/zarlink.o (sprintf)
E:/Program Files/Rowley Associates Limited/CrossWorks for ARM 1.3/lib/libc_v4t_a_ni_le.a(atoi.o)
                              ARM Flash Debug/i2cswitch.o (atoi)
E:/Program Files/Rowley Associates Limited/CrossWorks for ARM 1.3/lib/libc_v4t_a_ni_le.a(ctype.o)
                              E:/Program Files/Rowley Associates Limited/CrossWorks for ARM 1.3/lib/libc_v4t_a_ni_le.a(strtol.o) (isspace)
E:/Program Files/Rowley Associates Limited/CrossWorks for ARM 1.3/lib/libc_v4t_a_ni_le.a(__strtoul.o)
                              E:/Program Files/Rowley Associates Limited/CrossWorks for ARM 1.3/lib/libc_v4t_a_ni_le.a(strtol.o) (__strtoul)
E:/Program Files/Rowley Associates Limited/CrossWorks for ARM 1.3/lib/libc_v4t_a_ni_le.a(__digit.o)
                              E:/Program Files/Rowley Associates Limited/CrossWorks for ARM 1.3/lib/libc_v4t_a_ni_le.a(__strtoul.o) (__digit)
E:/Program Files/Rowley Associates Limited/CrossWorks for ARM 1.3/lib/lib_vfprintf_double_long_long_v4t_a_ni_le.a(__vfprintf_double_long_long.o)
                              E:/Program Files/Rowley Associates Limited/CrossWorks for ARM 1.3/lib/libc_v4t_a_ni_le.a(printf.o) (__vfprintf)
E:/Program Files/Rowley Associates Limited/CrossWorks for ARM 1.3/lib/libm_v4t_a_ni_le.a(__int64_to_float64.o)
                              E:/Program Files/Rowley Associates Limited/CrossWorks for ARM 1.3/lib/lib_vfprintf_double_long_long_v4t_a_ni_le.a(__vfprintf_double_long_long.o) (__floatdidf)
E:/Program Files/Rowley Associates Limited/CrossWorks for ARM 1.3/lib/libm_v4t_a_ni_le.a(__float32_to_int32.o)
                              E:/Program Files/Rowley Associates Limited/CrossWorks for ARM 1.3/lib/libm_v4t_a_ni_le.a(__int64_to_float64.o) (__float32_to_int32)
E:/Program Files/Rowley Associates Limited/CrossWorks for ARM 1.3/lib/libm_v4t_a_ni_le.a(__float32_to_int64.o)
                              E:/Program Files/Rowley Associates Limited/CrossWorks for ARM 1.3/lib/libm_v4t_a_ni_le.a(__int64_to_float64.o) (__float32_to_int64)
E:/Program Files/Rowley Associates Limited/CrossWorks for ARM 1.3/lib/libm_v4t_a_ni_le.a(__float32_to_uint32.o)
                              E:/Program Files/Rowley Associates Limited/CrossWorks for ARM 1.3/lib/libm_v4t_a_ni_le.a(__int64_to_float64.o) (__float32_to_uint32)
E:/Program Files/Rowley Associates Limited/CrossWorks for ARM 1.3/lib/libm_v4t_a_ni_le.a(__float32_to_uint64.o)
                              E:/Program Files/Rowley Associates Limited/CrossWorks for ARM 1.3/lib/libm_v4t_a_ni_le.a(__int64_to_float64.o) (__float32_to_uint64)
E:/Program Files/Rowley Associates Limited/CrossWorks for ARM 1.3/lib/libm_v4t_a_ni_le.a(__float32_to_float64.o)
                              E:/Program Files/Rowley Associates Limited/CrossWorks for ARM 1.3/lib/libm_v4t_a_ni_le.a(__int64_to_float64.o) (__float32_to_float64)
E:/Program Files/Rowley Associates Limited/CrossWorks for ARM 1.3/lib/libm_v4t_a_ni_le.a(__float64_to_int32.o)
                              E:/Program Files/Rowley Associates Limited/CrossWorks for ARM 1.3/lib/libm_v4t_a_ni_le.a(__int64_to_float64.o) (__float64_to_int32)
E:/Program Files/Rowley Associates Limited/CrossWorks for ARM 1.3/lib/libm_v4t_a_ni_le.a(__float64_to_int64.o)
                              E:/Program Files/Rowley Associates Limited/CrossWorks for ARM 1.3/lib/libm_v4t_a_ni_le.a(__int64_to_float64.o) (__float64_to_int64)
E:/Program Files/Rowley Associates Limited/CrossWorks for ARM 1.3/lib/libm_v4t_a_ni_le.a(__float64_to_uint32.o)
                              E:/Program Files/Rowley Associates Limited/CrossWorks for ARM 1.3/lib/libm_v4t_a_ni_le.a(__int64_to_float64.o) (__float64_to_uint32)
E:/Program Files/Rowley Associates Limited/CrossWorks for ARM 1.3/lib/libm_v4t_a_ni_le.a(__float64_to_uint64.o)
                              E:/Program Files/Rowley Associates Limited/CrossWorks for ARM 1.3/lib/lib_vfprintf_double_long_long_v4t_a_ni_le.a(__vfprintf_double_long_long.o) (__fixunsdfdi)
E:/Program Files/Rowley Associates Limited/CrossWorks for ARM 1.3/lib/libm_v4t_a_ni_le.a(__float64_to_float32.o)
                              E:/Program Files/Rowley Associates Limited/CrossWorks for ARM 1.3/lib/libm_v4t_a_ni_le.a(__int64_to_float64.o) (__float64_to_float32)
E:/Program Files/Rowley Associates Limited/CrossWorks for ARM 1.3/lib/libm_v4t_a_ni_le.a(frexp.o)
                              E:/Program Files/Rowley Associates Limited/CrossWorks for ARM 1.3/lib/lib_vfprintf_double_long_long_v4t_a_ni_le.a(__vfprintf_double_long_long.o) (frexp)
E:/Program Files/Rowley Associates Limited/CrossWorks for ARM 1.3/lib/libm_v4t_a_ni_le.a(ldexp.o)
                              E:/Program Files/Rowley Associates Limited/CrossWorks for ARM 1.3/lib/lib_vfprintf_double_long_long_v4t_a_ni_le.a(__vfprintf_double_long_long.o) (ldexp)
E:/Program Files/Rowley Associates Limited/CrossWorks for ARM 1.3/lib/libm_v4t_a_ni_le.a(__isinf.o)
                              E:/Program Files/Rowley Associates Limited/CrossWorks for ARM 1.3/lib/lib_vfprintf_double_long_long_v4t_a_ni_le.a(__vfprintf_double_long_long.o) (__isinf)
E:/Program Files/Rowley Associates Limited/CrossWorks for ARM 1.3/lib/libm_v4t_a_ni_le.a(__float64_infinity.o)
                              E:/Program Files/Rowley Associates Limited/CrossWorks for ARM 1.3/lib/libm_v4t_a_ni_le.a(ldexp.o) (__float64_infinity)
E:/Program Files/Rowley Associates Limited/CrossWorks for ARM 1.3/lib/libm_v4t_a_ni_le.a(__isnan.o)
                              E:/Program Files/Rowley Associates Limited/CrossWorks for ARM 1.3/lib/lib_vfprintf_double_long_long_v4t_a_ni_le.a(__vfprintf_double_long_long.o) (__isnan)
E:/Program Files/Rowley Associates Limited/CrossWorks for ARM 1.3/lib/libm_v4t_a_ni_le.a(__int32_to_float32.o)
                              E:/Program Files/Rowley Associates Limited/CrossWorks for ARM 1.3/lib/libm_v4t_a_ni_le.a(__int64_to_float64.o) (__int32_to_float32)
E:/Program Files/Rowley Associates Limited/CrossWorks for ARM 1.3/lib/libm_v4t_a_ni_le.a(__int32_to_float64.o)
                              E:/Program Files/Rowley Associates Limited/CrossWorks for ARM 1.3/lib/libm_v4t_a_ni_le.a(__int64_to_float64.o) (__int32_to_float64)
E:/Program Files/Rowley Associates Limited/CrossWorks for ARM 1.3/lib/libm_v4t_a_ni_le.a(__int64_to_float32.o)
                              E:/Program Files/Rowley Associates Limited/CrossWorks for ARM 1.3/lib/libm_v4t_a_ni_le.a(__int64_to_float64.o) (__int64_to_float32)
E:/Program Files/Rowley Associates Limited/CrossWorks for ARM 1.3/lib/libc_v4t_a_ni_le.a(__int64_umod.o)
                              E:/Program Files/Rowley Associates Limited/CrossWorks for ARM 1.3/lib/lib_vfprintf_double_long_long_v4t_a_ni_le.a(__vfprintf_double_long_long.o) (__umoddi3)
E:/Program Files/Rowley Associates Limited/CrossWorks for ARM 1.3/lib/libc_v4t_a_ni_le.a(__int64_lsl.o)
                              E:/Program Files/Rowley Associates Limited/CrossWorks for ARM 1.3/lib/libm_v4t_a_ni_le.a(__float32_to_int64.o) (__ashldi3)
E:/Program Files/Rowley Associates Limited/CrossWorks for ARM 1.3/lib/libc_v4t_a_ni_le.a(__int64_lsr.o)
                              E:/Program Files/Rowley Associates Limited/CrossWorks for ARM 1.3/lib/libm_v4t_a_ni_le.a(__float32_to_int64.o) (__lshrdi3)
E:/Program Files/Rowley Associates Limited/CrossWorks for ARM 1.3/lib/libc_v4t_a_ni_le.a(__int64_udivmod.o)
                              E:/Program Files/Rowley Associates Limited/CrossWorks for ARM 1.3/lib/lib_vfprintf_double_long_long_v4t_a_ni_le.a(__vfprintf_double_long_long.o) (__udivdi3)
E:/Program Files/Rowley Associates Limited/CrossWorks for ARM 1.3/lib/libc_v4t_a_ni_le.a(__int64_cmp.o)
                              E:/Program Files/Rowley Associates Limited/CrossWorks for ARM 1.3/lib/lib_vfprintf_double_long_long_v4t_a_ni_le.a(__vfprintf_double_long_long.o) (__cmpdi2)
E:/Program Files/Rowley Associates Limited/CrossWorks for ARM 1.3/lib/libc_v4t_a_ni_le.a(abs.o)
                              E:/Program Files/Rowley Associates Limited/CrossWorks for ARM 1.3/lib/lib_vfprintf_double_long_long_v4t_a_ni_le.a(__vfprintf_double_long_long.o) (abs)
E:/Program Files/Rowley Associates Limited/CrossWorks for ARM 1.3/lib/libc_v4t_a_ni_le.a(__pow10.o)
                              E:/Program Files/Rowley Associates Limited/CrossWorks for ARM 1.3/lib/lib_vfprintf_double_long_long_v4t_a_ni_le.a(__vfprintf_double_long_long.o) (__pow10)
E:/Program Files/Rowley Associates Limited/CrossWorks for ARM 1.3/lib/libc_v4t_a_ni_le.a(__hex_lc_uc.o)
                              E:/Program Files/Rowley Associates Limited/CrossWorks for ARM 1.3/lib/lib_vfprintf_double_long_long_v4t_a_ni_le.a(__vfprintf_double_long_long.o) (__hex_uc)

Allocating common symbols
Common symbol       size              file

uip_len             0x2               ARM Flash Debug/uip.o
errno               0x4               E:/Program Files/Rowley Associates Limited/CrossWorks for ARM 1.3/lib/libc_v4t_a_ni_le.a(errno.o)
hs                  0x4               ARM Flash Debug/httpd.o
uip_sappdata        0x4               ARM Flash Debug/uip.o
uip_acc32           0x4               ARM Flash Debug/uip.o
handlerTable        0x300             ARM Flash Debug/cli.o
uip_flags           0x1               ARM Flash Debug/uip.o
uip_appdata         0x4               ARM Flash Debug/uip.o
uip_conn            0x4               ARM Flash Debug/uip.o
uip_conns           0x320             ARM Flash Debug/uip.o
modulePresent       0x10              ARM Flash Debug/sfp.o
uip_listenports     0x28              ARM Flash Debug/uip.o
uip_stat            0x30              ARM Flash Debug/uip.o
uip_buf             0x5de             ARM Flash Debug/uip.o
uip_slen            0x2               ARM Flash Debug/uip.o

Memory Configuration

Name             Origin             Length             Attributes
Peripherals      0xe0000000         0x20000000         xw
SRAM             0x40000000         0x00010000         xw
FLASH            0x00000000         0x00020000         xr
*default*        0x00000000         0xffffffff

Linker script and memory map

                0xe0000000                __Peripherals_segment_start__ = 0xe0000000
                0x00000000                __Peripherals_segment_end__ = 0x0
                0x40000000                __SRAM_segment_start__ = 0x40000000
                0x40010000                __SRAM_segment_end__ = 0x40010000
                0x00000000                __FLASH_segment_start__ = 0x0
                0x00020000                __FLASH_segment_end__ = 0x20000

.vectors_ram    0x40000000       0x3c
                0x40000000                __vectors_ram_start__ = .
 *(.vectors_ram)
                0x4000003c                . = ((__vectors_ram_start__ + 0x3c) MAX_K .)
 *fill*         0x40000000       0x3c 00
                0x4000003c                __vectors_ram_end__ = (__vectors_ram_start__ + SIZEOF (.vectors_ram))
                0x00000001                . = ASSERT (((__vectors_ram_end__ >= __SRAM_segment_start__) && (__vectors_ram_end__ <= (__SRAM_segment_start__ + 0x10000))), .vectors_ram is too large to fit in SRAM memory segment)

.vectors        0x00000000       0x3c
                0x00000000                __vectors_start__ = .
 *(.vectors .vectors.*)
 .vectors       0x00000000       0x3c ARM Flash Debug/Philips_LPC210X_Startup.o
                0x0000003c                __vectors_end__ = (__vectors_start__ + SIZEOF (.vectors))
                0x00000001                . = ASSERT (((__vectors_end__ >= __FLASH_segment_start__) && (__vectors_end__ <= (__FLASH_segment_start__ + 0x20000))), .vectors is too large to fit in FLASH memory segment)

.init           0x0000003c      0x1e8
                0x0000003c                __init_start__ = .
 *(.init .init.*)
 .init          0x0000003c      0x1cc ARM Flash Debug/crt0.o
                0x0000003c                __start
                0x0000003c                _start
 .init          0x00000208       0x1c ARM Flash Debug/Philips_LPC210X_Startup.o
                0x0000020c                undef_handler
                0x00000214                pabort_handler
                0x00000218                dabort_handler
                0x00000210                swi_handler
                0x00000220                fiq_handler
                0x0000021c                irq_handler
                0x00000224                __init_end__ = (__init_start__ + SIZEOF (.init))
                0x00000001                . = ASSERT (((__init_end__ >= __FLASH_segment_start__) && (__init_end__ <= (__FLASH_segment_start__ + 0x20000))), .init is too large to fit in FLASH memory segment)

.text_load      0x00000224        0x0
                0x00000224                __text_load_start__ = .
 *(.text_load)
                0x00000224                __text_load_end__ = (__text_load_start__ + SIZEOF (.text_load))
                0x00000001                . = ASSERT (((__text_load_end__ >= __FLASH_segment_start__) && (__text_load_end__ <= (__FLASH_segment_start__ + 0x20000))), .text_load is too large to fit in FLASH memory segment)

.text           0x00000224    0x197ec
                0x00000224                __text_start__ = .
 *(.text .text.* .glue_7t .glue_7 .gnu.linkonce.t.*)
 .text          0x00000224      0x2bc ARM Flash Debug/zarlink.o
                0x00000224                zarlinkInit
 .text          0x000004e0      0x444 ARM Flash Debug/armvic.o
                0x000006d0                armvicIntConnect
                0x00000780                armvicIntDisconnect
                0x00000594                armvicInit
                0x0000081c                armvicSoftIntNegate
                0x00000854                armvicIntEnable
                0x000008bc                armvicIntDisable
                0x000007fc                armvicSoftIntAssert
                0x00000630                armvicInit2
                0x0000083c                armvicSoftIntNegateAll
                0x00000660                armvicIntPrioLevelSet
 .text          0x00000924      0x27c ARM Flash Debug/board.o
                0x00000944                boardSetTimerLed
                0x00000964                boardTimerLedToggle
                0x00000924                boardSetBusyLed
                0x000009bc                boardInit2
                0x000009a8                boardInit
 .text          0x00000ba0      0x7b8 ARM Flash Debug/cli.o
                0x0000101c                cliRegisterCommand
                0x0000121c                helpHandler
                0x00000fd8                cliInit
                0x000010cc                cliDoCommand
 .text          0x00001358      0x6cc ARM Flash Debug/clichar.o
                0x0000180c                echoHandler
                0x0000149c                clicharSendOutputBuffer
                0x00001770                clicharEventTrigger
                0x0000196c                clicharInit
                0x00001478                clicharPuts
                0x000013a0                clicharGetOutputBuffer
 .text          0x00001a24      0x120 ARM Flash Debug/clivar.o
                0x00001abc                addVariableHandler
                0x00001a24                clivarInit
 .text          0x00001b44      0x1d0 ARM Flash Debug/crc16.o
                0x00001b60                crc16Update
                0x00001b44                crc16Init
                0x00001c70                crc16Calc
                0x00001bcc                crc16StrUpdate
 .text          0x00001d14      0xb18 ARM Flash Debug/ee24lc256.o
                0x00001e30                ee24lc256ReadByte
                0x000022e0                ee24lc256AckPoll
                0x00002178                ee24lc256GetDeviceInfo
                0x0000203c                ee24lc256WritePage
                0x00001ef0                ee24lc256ReadPage
                0x00001d78                ee24lc256WriteByte
                0x000021e0                ee24lc256Init
 .text          0x0000282c      0x58c ARM Flash Debug/eventq.o
                0x0000282c                eventqInit
                0x00002d0c                eventqDispatch
                0x00002c88                eventqGetHandler
                0x00002ab8                eventqGet
                0x00002c20                eventqRegisterHandler
                0x000028f8                eventqPut
                0x000029d4                eventqUrgentPut
 .text          0x00002db8      0xfa4 ARM Flash Debug/i2cmaster.o
                0x000038f4                i2cmasterProbe
                0x00003c2c                i2cmasterSendOne
                0x0000352c                i2cmasterInit
                0x00003664                i2cmasterPut
                0x00003a60                i2cmasterReceive
                0x00003b4c                i2cmasterSend
                0x000037ac                i2cmasterGet
                0x00003ca0                i2cmasterSendMult
                0x00003778                i2cmasterGetData
 .text          0x00003d5c      0x608 ARM Flash Debug/i2cport.o
                0x00004030                i2cportAssign
                0x00003f18                i2cportInit
                0x00004110                i2cportClear
                0x00003ff0                i2cportDirConfig
                0x0000408c                i2cportSet
                0x00004198                i2cportGet
 .text          0x00004364      0x264 ARM Flash Debug/i2cswitch.o
                0x000043c4                i2cswitchSetBus
                0x00004364                i2cswitchInit
                0x00004444                i2cswitchDisable
 .text          0x000045c8      0x2a0 ARM Flash Debug/init.o
                0x000045c8                main
 .text          0x00004868      0x18c ARM Flash Debug/medusa.o
                0x0000493c                medusaToggleGreenLed
                0x0000496c                medusaSetOrangeLed
                0x000048e4                medusaSetGreenLed
                0x000049c4                medusaToggleOrangeLed
                0x00004868                medusaInit
 .text          0x000049f4      0x2a8 ARM Flash Debug/pll.o
                0x00004b38                pllSetPeriphDivider
                0x000049f4                pllInit
                0x00004c48                pllGetPeriphFreq
                0x00004c28                pllGetCpuFreq
                0x00004c7c                pllGetPeriphDivider
 .text          0x00004c9c      0xda0 ARM Flash Debug/sfpdiag.o
                0x00005340                sfpdiagSoftRxRateSelect
                0x0000546c                sfpdiagRetrieveInfoRaw
                0x00005178                sfpdiagGetWavelength
                0x00005430                sfpdiagRetrieveInfo
                0x00004c9c                sfpdiagInit
                0x0000503c                sfpdiagGetDiags
                0x00005250                sfpdiagSoftTxDisable
 .text          0x00005a3c      0x850 ARM Flash Debug/spi.o
                0x00005a3c                spiPut
                0x00006138                spiInit
                0x00005b6c                spiGet
 .text          0x0000628c      0x2e8 ARM Flash Debug/timer0.o
                0x000064f4                timer0Delay
                0x0000628c                timer0Init
                0x00006554                timer0GetTicks
 .text          0x00006574      0xa38 ARM Flash Debug/uart0.o
                0x00006f70                __putchar
                0x00006860                uart0Init2
                0x0000677c                uart0Init
                0x00006890                uart0Puts
                0x00006b94                uart0RxOne
                0x00006920                uart0TxOne
 .text          0x00006fac      0x110 ARM Flash Debug/watchdog.o
                0x0000705c                watchdogInit
                0x00006fac                watchdogKick
 .text          0x000070bc      0x604 ARM Flash Debug/sfp.o
                0x000072b4                sfpEnable
                0x00007168                sfpModulePresent
                0x00007238                sfpTransmitDisable
                0x000070bc                sfpInit
                0x000071d4                sfpProbe
 .text          0x000076c0      0x24c ARM Flash Debug/strutil.o
                0x000077a4                strutilHexdump
                0x000076c0                strutil_strncasecmp
 .text          0x0000790c      0x49c ARM Flash Debug/zl_ssi.o
 .text          0x00007da8     0x30a0 ARM Flash Debug/zl_rmon.o
                0x0000a118                zarlinkRmonInit
                0x0000a188                zarlinkRmonUpdateStats
                0x0000a278                zarlinkRmonCounterOverflow
                0x000089d4                zarlinkRmonGet
 .text          0x0000ae48      0x8ec ARM Flash Debug/zl_frame.o
                0x0000b4e8                zarlinkEthFrameRead
                0x0000ae48                zarlinkEthFrameWrite
 .text          0x0000b734      0xba0 ARM Flash Debug/zl_mii.o
                0x0000b734                zarlinkMiiWrite
                0x0000b884                zarlinkMiiRead
                0x0000ba68                zarlinkMiiDump
                0x0000c284                zarlinkMiiInit
                0x0000bba4                zarlinkMiiPowerSave
                0x0000bc6c                zarlinkForceMiiPowerSave
 .text          0x0000c2d4      0x580 ARM Flash Debug/zl_bus.o
                0x0000c684                zarlinkFrameWrite8
                0x0000c574                zarlinkIndexedWrite
                0x0000c6f8                zarlinkFrameRead8
                0x0000c750                zarlinkCtrlBuffer1Write
                0x0000c6b0                zarlinkFrameWrite
                0x0000c800                zarlinkInterruptWrite
                0x0000c660                zarlinkStatusRead
                0x0000c7cc                zarlinkCtrlBuffer2Read
                0x0000c71c                zarlinkFrameRead
                0x0000c5d8                zarlinkIndexedRead
                0x0000c830                zarlinkInterruptRead
                0x0000c798                zarlinkCtrlBuffer1Read
                0x0000c634                zarlinkCommandWrite
 .text          0x0000c854     0x1138 ARM Flash Debug/zl_util.o
                0x0000c89c                swapMac
                0x0000d1e4                zarlinkCpuMacAddrGet
                0x0000c934                parseDottedQuadV4
                0x0000d0f8                zarlinkCpuMacAddrSetUip
                0x0000d898                zarlinkUtilInit
                0x0000c854                byteSwap16
                0x0000d068                zarlinkCpuMacAddrSet
 .text          0x0000d98c      0x6b8 ARM Flash Debug/zl_mirror.o
                0x0000dfa0                zarlinkMirrorInit
 .text          0x0000e044      0x680 ARM Flash Debug/zl_event.o
                0x0000e504                zarlinkEventUnmaskIrq
                0x0000e4b4                zarlinkEventMaskIrq
                0x0000e044                zarlinkEventInit
                0x0000e55c                zarlinkEventMaskPorts
 .text          0x0000e6c4      0x620 ARM Flash Debug/icmp.o
                0x0000e9b0                icmpArpRequestSend
                0x0000ecb0                icmpInit
                0x0000ea04                icmpArpReplySend
 .text          0x0000ece4      0x158 ARM Flash Debug/pm.o
                0x0000edd4                pmIdle
                0x0000ed10                pmInit
                0x0000ed6c                pmSleep
 .text          0x0000ee3c      0x1bc ARM Flash Debug/armirq.o
                0x0000eeb8                restoreIRQ
                0x0000efc0                enableFIQ
                0x0000ef3c                disableFIQ
                0x0000ef04                enableIRQ
                0x0000ef74                restoreFIQ
                0x0000ee3c                disableIRQ
 .text          0x0000eff8      0x2d8 ARM Flash Debug/zl_ctrl1.o
                0x0000f204                zarlinkCtrlRetrieveCtrl1
                0x0000f2a8                zarlinkCtrl1Init
 .text          0x0000f2d0       0xcc ARM Flash Debug/zl_ctrl2.o
                0x0000f374                zarlinkCtrl2Init
                0x0000f2d0                zarlinkCtrlRetrieveCtrl2
 .text          0x0000f39c       0x70 ARM Flash Debug/zl_reset.o
                0x0000f3e4                zarlinkResetInit
 .text          0x0000f40c      0x194 ARM Flash Debug/ip.o
                0x0000f56c                ipInit
                0x0000f4e4                ipAddrGet
 .text          0x0000f5a0     0x1164 ARM Flash Debug/nvstore.o
                0x0000fa3c                nvstoreInit
                0x0000fb98                nvstoreWrite
                0x0000ffe0                nvstoreRead
 .text          0x00010704      0x134 ARM Flash Debug/zl_rxframe.o
                0x00010810                zarlinkRxFrameInit
 .text          0x00010838      0x210 ARM Flash Debug/trunk.o
                0x00010914                trunkInit
                0x00010860                trunkTeardown
                0x00010838                trunkBuild
 .text          0x00010a48      0x97c ARM Flash Debug/uip_arp.o
                0x000110e4                uip_arp_out
                0x00010f2c                uip_arp_arpin
                0x00010ac4                uip_arp_timer
                0x00010a48                uip_arp_init
                0x00010e5c                uip_arp_ipin
 .text          0x000113c4      0x524 ARM Flash Debug/cgi.o
 .text          0x000118e8      0x2a4 ARM Flash Debug/fs.o
                0x000119b0                fs_open
                0x00011a94                fs_init
                0x00011ae8                fs_count
 .text          0x00011b8c      0x840 ARM Flash Debug/httpd.o
                0x00011b8c                httpd_init
                0x00011ba8                httpd_appcall
 .text          0x000123cc      0x1ec ARM Flash Debug/memb.o
                0x00012410                memb_alloc
                0x000124bc                memb_free
                0x000123cc                memb_init
                0x0001256c                memb_ref
 .text          0x000125b8      0x970 ARM Flash Debug/telnetd.o
                0x0001271c                telnetd_output
                0x00012ce0                telnetd_app
                0x0001283c                telnetd_init
                0x000126c8                telnetd_prompt
                0x000126a4                telnetd_close
 .text          0x00012f28      0x594 ARM Flash Debug/telnetd-shell.o
                0x00013478                telnetd_input
                0x00013424                telnetd_connected
 .text          0x000134bc     0x23f0 ARM Flash Debug/uip.o
                0x00013900                uip_unlisten
                0x00013ad4                uip_process
                0x000139a4                uip_listen
                0x00013604                uip_connect
                0x00015868                htons
                0x000134bc                uip_init
 .text          0x000158ac      0x52c ARM Flash Debug/uip_arch.o
                0x000158ac                uip_add32
                0x00015b60                uip_ipchksum
                0x00015b90                uip_tcpchksum
                0x00015a34                uip_chksum
 .text          0x00015dd8      0x6ec E:/Program Files/Rowley Associates Limited/CrossWorks for ARM 1.3/lib/libm_v4t_a_ni_le.a(sf-wrapper.o)
                0x00016188                __divsf3
                0x00016400                __fixsfsi
                0x00015de0                __subsf3
                0x00016330                __lesf2
                0x00016338                __nesf2
                0x00016328                __gtsf2
                0x00015fac                __floatsisf
                0x00016338                __eqsf2
                0x00015dd8                __negsf2
                0x00016338                __cmpsf2
                0x00016330                __ltsf2
                0x00015ff8                __mulsf3
                0x00016328                __gesf2
                0x000163c4                __unordsf2
                0x00015fa4                __floatunsisf
                0x00016468                __fixunssfsi
                0x00015de4                __addsf3
 .text          0x000164c4      0xb28 E:/Program Files/Rowley Associates Limited/CrossWorks for ARM 1.3/lib/libm_v4t_a_ni_le.a(df-wrapper.o)
                0x00016d28                __cmpdf2
                0x00016d28                __eqdf2
                0x00016d18                __gtdf2
                0x000167dc                __floatsidf
                0x00016d20                __ltdf2
                0x00016e80                __fixunsdfsi
                0x00016808                __extendsfdf2
                0x000164d0                __adddf3
                0x000167b4                __floatunsidf
                0x00016e00                __fixdfsi
                0x00016d20                __ledf2
                0x000164c4                __negdf2
                0x00016aac                __divdf3
                0x00016854                __muldf3
                0x00016ef4                __truncdfsf2
                0x00016d28                __nedf2
                0x00016dbc                __unorddf2
                0x00016d18                __gedf2
                0x000164cc                __subdf3
 .text          0x00016fec       0x30 E:/Program Files/Rowley Associates Limited/CrossWorks for ARM 1.3/lib/libc_v4t_a_ni_le.a(__int32_udivmod.o)
                0x00016fec                __int32_udiv
                0x00016fec                __int32_udivmod
                0x00016fec                __udivsi3
 .text          0x0001701c       0x18 E:/Program Files/Rowley Associates Limited/CrossWorks for ARM 1.3/lib/libc_v4t_a_ni_le.a(strlen.o)
                0x0001701c                strlen
 .text          0x00017034       0x54 E:/Program Files/Rowley Associates Limited/CrossWorks for ARM 1.3/lib/libc_v4t_a_ni_le.a(memcpy.o)
                0x00017034                memcpy
 .text          0x00017088       0x94 E:/Program Files/Rowley Associates Limited/CrossWorks for ARM 1.3/lib/libc_v4t_a_ni_le.a(memset.o)
                0x00017088                memset
 .text          0x0001711c       0x58 E:/Program Files/Rowley Associates Limited/CrossWorks for ARM 1.3/lib/libc_v4t_a_ni_le.a(strncpy.o)
                0x0001711c                strncpy
 .text          0x00017174       0xc8 E:/Program Files/Rowley Associates Limited/CrossWorks for ARM 1.3/lib/libc_v4t_a_ni_le.a(strtol.o)
                0x00017174                strtol
 .text          0x0001723c       0x48 E:/Program Files/Rowley Associates Limited/CrossWorks for ARM 1.3/lib/libc_v4t_a_ni_le.a(printf.o)
                0x0001723c                printf
 .text          0x00017284       0x40 E:/Program Files/Rowley Associates Limited/CrossWorks for ARM 1.3/lib/libc_v4t_a_ni_le.a(sprintf.o)
                0x00017284                sprintf
 .text          0x000172c4       0x2c E:/Program Files/Rowley Associates Limited/CrossWorks for ARM 1.3/lib/libc_v4t_a_ni_le.a(atoi.o)
                0x000172c4                atoi
 .text          0x000172f0      0x1cc E:/Program Files/Rowley Associates Limited/CrossWorks for ARM 1.3/lib/libc_v4t_a_ni_le.a(ctype.o)
                0x000174a8                isblank
                0x00017320                islower
                0x00017474                tolower
                0x00017394                ispunct
                0x00017378                isspace
                0x00017348                isxdigit
                0x0001730c                isupper
                0x000172f0                isalpha
                0x00017414                isgraph
                0x000173d0                isalnum
                0x00017400                isprint
                0x00017334                isdigit
                0x00017460                iscntrl
                0x00017494                toupper
 .text          0x000174bc      0x128 E:/Program Files/Rowley Associates Limited/CrossWorks for ARM 1.3/lib/libc_v4t_a_ni_le.a(__strtoul.o)
                0x000174bc                __strtoul
 .text          0x000175e4       0x5c E:/Program Files/Rowley Associates Limited/CrossWorks for ARM 1.3/lib/libc_v4t_a_ni_le.a(__digit.o)
                0x000175e4                __digit
 .text          0x00017640     0x172c E:/Program Files/Rowley Associates Limited/CrossWorks for ARM 1.3/lib/lib_vfprintf_double_long_long_v4t_a_ni_le.a(__vfprintf_double_long_long.o)
                0x000176fc                __vfprintf
 .text          0x00018d6c      0x178 E:/Program Files/Rowley Associates Limited/CrossWorks for ARM 1.3/lib/libm_v4t_a_ni_le.a(__int64_to_float64.o)
                0x00018d6c                __floatdidf
                0x00018d6c                __int64_to_float64
 .text          0x00018ee4       0x40 E:/Program Files/Rowley Associates Limited/CrossWorks for ARM 1.3/lib/libm_v4t_a_ni_le.a(__float32_to_int32.o)
                0x00018ee4                __float32_to_int32
 .text          0x00018f24       0x84 E:/Program Files/Rowley Associates Limited/CrossWorks for ARM 1.3/lib/libm_v4t_a_ni_le.a(__float32_to_int64.o)
                0x00018f24                __float32_to_int64
                0x00018f24                __fixsfdi
 .text          0x00018fa8       0x40 E:/Program Files/Rowley Associates Limited/CrossWorks for ARM 1.3/lib/libm_v4t_a_ni_le.a(__float32_to_uint32.o)
                0x00018fa8                __float32_to_uint32
 .text          0x00018fe8       0x84 E:/Program Files/Rowley Associates Limited/CrossWorks for ARM 1.3/lib/libm_v4t_a_ni_le.a(__float32_to_uint64.o)
                0x00018fe8                __float32_to_uint64
                0x00018fe8                __fixunssfdi
 .text          0x0001906c       0x6c E:/Program Files/Rowley Associates Limited/CrossWorks for ARM 1.3/lib/libm_v4t_a_ni_le.a(__float32_to_float64.o)
                0x0001906c                __float32_to_float64
 .text          0x000190d8       0x80 E:/Program Files/Rowley Associates Limited/CrossWorks for ARM 1.3/lib/libm_v4t_a_ni_le.a(__float64_to_int32.o)
                0x000190d8                __float64_to_int32
 .text          0x00019158       0xb0 E:/Program Files/Rowley Associates Limited/CrossWorks for ARM 1.3/lib/libm_v4t_a_ni_le.a(__float64_to_int64.o)
                0x00019158                __float64_to_int64
                0x00019158                __fixdfdi
 .text          0x00019208       0x7c E:/Program Files/Rowley Associates Limited/CrossWorks for ARM 1.3/lib/libm_v4t_a_ni_le.a(__float64_to_uint32.o)
                0x00019208                __float64_to_uint32
 .text          0x00019284       0xac E:/Program Files/Rowley Associates Limited/CrossWorks for ARM 1.3/lib/libm_v4t_a_ni_le.a(__float64_to_uint64.o)
                0x00019284                __fixunsdfdi
                0x00019284                __float64_to_uint64
 .text          0x00019330       0x58 E:/Program Files/Rowley Associates Limited/CrossWorks for ARM 1.3/lib/libm_v4t_a_ni_le.a(__float64_to_float32.o)
                0x00019330                __float64_to_float32
 .text          0x00019388       0x90 E:/Program Files/Rowley Associates Limited/CrossWorks for ARM 1.3/lib/libm_v4t_a_ni_le.a(frexp.o)
                0x00019388                frexp
 .text          0x00019418       0xc0 E:/Program Files/Rowley Associates Limited/CrossWorks for ARM 1.3/lib/libm_v4t_a_ni_le.a(ldexp.o)
                0x00019418                ldexp
 .text          0x000194d8       0x40 E:/Program Files/Rowley Associates Limited/CrossWorks for ARM 1.3/lib/libm_v4t_a_ni_le.a(__isinf.o)
                0x000194d8                __isinf
 .text          0x00019518       0x48 E:/Program Files/Rowley Associates Limited/CrossWorks for ARM 1.3/lib/libm_v4t_a_ni_le.a(__isnan.o)
                0x00019518                __isnan
 .text          0x00019560       0xb8 E:/Program Files/Rowley Associates Limited/CrossWorks for ARM 1.3/lib/libm_v4t_a_ni_le.a(__int32_to_float32.o)
                0x00019560                __int32_to_float32
 .text          0x00019618       0xd8 E:/Program Files/Rowley Associates Limited/CrossWorks for ARM 1.3/lib/libm_v4t_a_ni_le.a(__int32_to_float64.o)
                0x00019618                __int32_to_float64
 .text          0x000196f0      0x18c E:/Program Files/Rowley Associates Limited/CrossWorks for ARM 1.3/lib/libm_v4t_a_ni_le.a(__int64_to_float32.o)
                0x000196f0                __int64_to_float32
                0x000196f0                __floatdisf
 .text          0x0001987c       0x18 E:/Program Files/Rowley Associates Limited/CrossWorks for ARM 1.3/lib/libc_v4t_a_ni_le.a(__int64_umod.o)
                0x0001987c                __int64_umod
                0x0001987c                __umoddi3
 .text          0x00019894       0x28 E:/Program Files/Rowley Associates Limited/CrossWorks for ARM 1.3/lib/libc_v4t_a_ni_le.a(__int64_lsl.o)
                0x00019894                __ashldi3
                0x00019894                __int64_lsl
 .text          0x000198bc       0x2c E:/Program Files/Rowley Associates Limited/CrossWorks for ARM 1.3/lib/libc_v4t_a_ni_le.a(__int64_lsr.o)
                0x000198bc                __int64_lsr
                0x000198bc                __lshrdi3
 .text          0x000198e8       0x68 E:/Program Files/Rowley Associates Limited/CrossWorks for ARM 1.3/lib/libc_v4t_a_ni_le.a(__int64_udivmod.o)
                0x000198e8                __int64_udivmod
                0x000198e8                __int64_udiv
                0x000198e8                __udivdi3
 .text          0x00019950       0x24 E:/Program Files/Rowley Associates Limited/CrossWorks for ARM 1.3/lib/libc_v4t_a_ni_le.a(__int64_cmp.o)
                0x00019950                __cmpdi2
                0x00019950                __int64_cmp
 .text          0x00019974        0xc E:/Program Files/Rowley Associates Limited/CrossWorks for ARM 1.3/lib/libc_v4t_a_ni_le.a(abs.o)
                0x00019974                abs
 .text          0x00019980       0x90 E:/Program Files/Rowley Associates Limited/CrossWorks for ARM 1.3/lib/libc_v4t_a_ni_le.a(__pow10.o)
                0x00019980                __pow10
                0x00019a10                __text_end__ = (__text_start__ + SIZEOF (.text))
                0x00000001                . = ASSERT (((__text_end__ >= __FLASH_segment_start__) && (__text_end__ <= (__FLASH_segment_start__ + 0x20000))), .text is too large to fit in FLASH memory segment)

.dtors          0x00019a10        0x0
                0x00019a10                __dtors_start__ = .
 *(SORT(.dtors.*))
 *(.dtors)
                0x00019a10                __dtors_end__ = (__dtors_start__ + SIZEOF (.dtors))
                0x00000001                . = ASSERT (((__dtors_end__ >= __FLASH_segment_start__) && (__dtors_end__ <= (__FLASH_segment_start__ + 0x20000))), .dtors is too large to fit in FLASH memory segment)

.ctors          0x00019a10        0x0
                0x00019a10                __ctors_start__ = .
 *(SORT(.ctors.*))
 *(.ctors)
                0x00019a10                __ctors_end__ = (__ctors_start__ + SIZEOF (.ctors))
                0x00000001                . = ASSERT (((__ctors_end__ >= __FLASH_segment_start__) && (__ctors_end__ <= (__FLASH_segment_start__ + 0x20000))), .ctors is too large to fit in FLASH memory segment)

.rodata         0x00019a10     0x3628
                0x00019a10                __rodata_start__ = .
 *(.rodata .rodata.* .gnu.linkonce.r.*)
 .rodata        0x00019a10       0x30 ARM Flash Debug/zarlink.o
 .rodata        0x00019a40       0x40 ARM Flash Debug/armvic.o
 .rodata        0x00019a80       0x80 ARM Flash Debug/board.o
 .rodata        0x00019b00       0x60 ARM Flash Debug/cli.o
 .rodata        0x00019b60       0x60 ARM Flash Debug/clichar.o
 .rodata        0x00019bc0       0x40 ARM Flash Debug/clivar.o
 .rodata        0x00019c00      0x1f8 ARM Flash Debug/ee24lc256.o
 .rodata        0x00019df8       0xbc ARM Flash Debug/i2cport.o
 .rodata        0x00019eb4       0xc0 ARM Flash Debug/i2cswitch.o
 .rodata        0x00019f74       0x68 ARM Flash Debug/init.o
 .rodata        0x00019fdc      0x1d8 ARM Flash Debug/sfpdiag.o
 .rodata        0x0001a1b4       0xfc ARM Flash Debug/spi.o
 .rodata        0x0001a2b0       0x8c ARM Flash Debug/uart0.o
 .rodata        0x0001a33c       0x34 ARM Flash Debug/watchdog.o
 .rodata        0x0001a370      0x1e8 ARM Flash Debug/sfp.o
 .rodata        0x0001a558       0x14 ARM Flash Debug/strutil.o
 .rodata        0x0001a56c      0x2cc ARM Flash Debug/zl_rmon.o
 .rodata        0x0001a838      0x380 ARM Flash Debug/zl_mii.o
 .rodata        0x0001abb8      0x430 ARM Flash Debug/zl_util.o
 .rodata        0x0001afe8       0xc0 ARM Flash Debug/zl_mirror.o
 .rodata        0x0001b0a8       0xc4 ARM Flash Debug/zl_event.o
 .rodata        0x0001b16c       0xc8 ARM Flash Debug/icmp.o
 .rodata        0x0001b234       0x28 ARM Flash Debug/pm.o
 .rodata        0x0001b25c       0x3c ARM Flash Debug/zl_ctrl1.o
 .rodata        0x0001b298       0x20 ARM Flash Debug/zl_reset.o
 .rodata        0x0001b2b8       0x50 ARM Flash Debug/ip.o
 .rodata        0x0001b308      0x160 ARM Flash Debug/nvstore.o
 .rodata        0x0001b468       0x3c ARM Flash Debug/trunk.o
 .rodata        0x0001b4a4      0x11c ARM Flash Debug/cgi.o
 .rodata        0x0001b5c0     0x1668 ARM Flash Debug/fs.o
                0x0001cbc4                file_index_html
                0x0001cb4c                file_img_bg_png
                0x0001cb10                file_cgi_files
                0x0001cbec                file_stats_header_html
                0x0001cb88                file_404_html
                0x0001cb74                file_control_html
                0x0001cb60                file_about_html
                0x0001cc00                file_tcp_footer_plain
                0x0001cb24                file_cgi_stats
                0x0001cbb0                file_files_header_html
                0x0001cb38                file_cgi_tcp
                0x0001cbd8                file_stats_footer_plain
                0x0001cb9c                file_files_footer_plain
                0x0001cc14                file_tcp_header_html
 .rodata        0x0001cc28       0x44 ARM Flash Debug/telnetd.o
 .rodata        0x0001cc6c      0x1a4 ARM Flash Debug/telnetd-shell.o
 .rodata        0x0001ce10        0xc ARM Flash Debug/uip.o
                0x0001ce18                uip_arp_netmask
                0x0001ce10                uip_hostaddr
                0x0001ce14                uip_arp_draddr
 .rodata        0x0001ce1c      0x100 E:/Program Files/Rowley Associates Limited/CrossWorks for ARM 1.3/lib/libc_v4t_a_ni_le.a(ctype.o)
                0x0001ce1c                __ctype
 .rodata        0x0001cf1c       0x98 E:/Program Files/Rowley Associates Limited/CrossWorks for ARM 1.3/lib/lib_vfprintf_double_long_long_v4t_a_ni_le.a(__vfprintf_double_long_long.o)
 .rodata.str1.4
                0x0001cfb4       0x12 E:/Program Files/Rowley Associates Limited/CrossWorks for ARM 1.3/lib/lib_vfprintf_double_long_long_v4t_a_ni_le.a(__vfprintf_double_long_long.o)
                                 0x14 (size before relaxing)
 *fill*         0x0001cfc6        0x2 00
 .rodata        0x0001cfc8        0x8 E:/Program Files/Rowley Associates Limited/CrossWorks for ARM 1.3/lib/libm_v4t_a_ni_le.a(__float64_infinity.o)
                0x0001cfc8                __float64_infinity
 .rodata        0x0001cfd0       0x48 E:/Program Files/Rowley Associates Limited/CrossWorks for ARM 1.3/lib/libc_v4t_a_ni_le.a(__pow10.o)
 .rodata        0x0001d018       0x20 E:/Program Files/Rowley Associates Limited/CrossWorks for ARM 1.3/lib/libc_v4t_a_ni_le.a(__hex_lc_uc.o)
                0x0001d018                __hex_uc
                0x0001d028                __hex_lc
                0x0001d038                __rodata_end__ = (__rodata_start__ + SIZEOF (.rodata))
                0x00000001                . = ASSERT (((__rodata_end__ >= __FLASH_segment_start__) && (__rodata_end__ <= (__FLASH_segment_start__ + 0x20000))), .rodata is too large to fit in FLASH memory segment)
                0x0001d038                __fast_load_start__ = (((__rodata_end__ + 0x3) / 0x4) * 0x4)

.fast           0x4000003c        0x0 load address 0x0001d038
                0x4000003c                __fast_start__ = .
 *(.fast .fast.*)
                0x4000003c                __fast_end__ = (__fast_start__ + SIZEOF (.fast))
                0x00000001                . = ASSERT ((((__fast_load_start__ + SIZEOF (.fast)) >= __FLASH_segment_start__) && ((__fast_load_start__ + SIZEOF (.fast)) <= (__FLASH_segment_start__ + 0x20000))), .fast is too large to fit in FLASH memory segment)

.fast_run       0x4000003c        0x0
                0x4000003c                __fast_run_start__ = .
                0x4000003c                . = ((__fast_run_start__ + SIZEOF (.fast)) MAX_K .)
                0x4000003c                __fast_run_end__ = (__fast_run_start__ + SIZEOF (.fast_run))
                0x00000001                . = ASSERT (((__fast_run_end__ >= __SRAM_segment_start__) && (__fast_run_end__ <= (__SRAM_segment_start__ + 0x10000))), .fast_run is too large to fit in SRAM memory segment)
                0x0001d038                __data_load_start__ = ((((__fast_load_start__ + SIZEOF (.fast)) + 0x3) / 0x4) * 0x4)

.data           0x4000003c      0x430 load address 0x0001d038
                0x4000003c                __data_start__ = .
 *(.data .data.* .gnu.linkonce.d.*)
 .data          0x4000003c        0x6 ARM Flash Debug/clichar.o
 *fill*         0x40000042        0x2 00
 .data          0x40000044        0x4 ARM Flash Debug/clivar.o
 .data          0x40000048      0x200 ARM Flash Debug/crc16.o
 .data          0x40000248        0x2 ARM Flash Debug/i2cport.o
 *fill*         0x4000024a        0x2 00
 .data          0x4000024c       0x1c ARM Flash Debug/init.o
                0x40000260                cpuMacAddr
 .data          0x40000268        0xc ARM Flash Debug/pll.o
 .data          0x40000274       0x20 ARM Flash Debug/uart0.o
 .data          0x40000294      0x100 ARM Flash Debug/strutil.o
 .data          0x40000394       0x64 ARM Flash Debug/zl_mii.o
 .data          0x400003f8       0x10 ARM Flash Debug/zl_util.o
 .data          0x40000408        0x4 ARM Flash Debug/ip.o
 .data          0x4000040c        0x6 ARM Flash Debug/uip_arp.o
                0x4000040c                uip_ethaddr
 *fill*         0x40000412        0x2 00
 .data          0x40000414       0x30 ARM Flash Debug/cgi.o
                0x40000414                cgitab
 .data          0x40000444        0x8 ARM Flash Debug/telnetd.o
 .data          0x4000044c       0x20 ARM Flash Debug/telnetd-shell.o
                0x4000046c                __data_end__ = (__data_start__ + SIZEOF (.data))
                0x00000001                . = ASSERT ((((__data_load_start__ + SIZEOF (.data)) >= __FLASH_segment_start__) && ((__data_load_start__ + SIZEOF (.data)) <= (__FLASH_segment_start__ + 0x20000))), .data is too large to fit in FLASH memory segment)

.data_run       0x4000003c      0x430
                0x4000003c                __data_run_start__ = .
                0x4000046c                . = ((__data_run_start__ + SIZEOF (.data)) MAX_K .)
 *fill*         0x4000003c      0x430 00
                0x4000046c                __data_run_end__ = (__data_run_start__ + SIZEOF (.data_run))
                0x00000001                . = ASSERT (((__data_run_end__ >= __SRAM_segment_start__) && (__data_run_end__ <= (__SRAM_segment_start__ + 0x10000))), .data_run is too large to fit in SRAM memory segment)

.bss            0x4000046c     0x2530
                0x4000046c                __bss_start__ = .
 *(.bss .bss.* .gnu.linkonce.b.*)
 .bss           0x4000046c        0x4 ARM Flash Debug/armvic.o
 .bss           0x40000470       0xa4 ARM Flash Debug/cli.o
 .bss           0x40000514      0x20c ARM Flash Debug/clichar.o
 .bss           0x40000720      0x284 ARM Flash Debug/clivar.o
 .bss           0x400009a4       0x41 ARM Flash Debug/ee24lc256.o
 *fill*         0x400009e5        0x3 00
 .bss           0x400009e8       0xcc ARM Flash Debug/eventq.o
 .bss           0x40000ab4      0x240 ARM Flash Debug/i2cmaster.o
 .bss           0x40000cf4        0x8 ARM Flash Debug/i2cport.o
 .bss           0x40000cfc        0x1 ARM Flash Debug/i2cswitch.o
 .bss           0x40000cfd       0x80 ARM Flash Debug/init.o
 *fill*         0x40000d7d        0x3 00
 .bss           0x40000d80        0x8 ARM Flash Debug/medusa.o
 .bss           0x40000d88        0x4 ARM Flash Debug/pll.o
 .bss           0x40000d8c       0xc8 ARM Flash Debug/sfpdiag.o
 .bss           0x40000e54       0xd0 ARM Flash Debug/spi.o
 .bss           0x40000f24       0x10 ARM Flash Debug/timer0.o
 .bss           0x40000f34      0x190 ARM Flash Debug/uart0.o
 .bss           0x400010c4      0x988 ARM Flash Debug/zl_rmon.o
 .bss           0x40001a4c        0xc ARM Flash Debug/zl_frame.o
                0x40001a4c                frameDataReady
 .bss           0x40001a58       0x2c ARM Flash Debug/zl_util.o
 .bss           0x40001a84       0x20 ARM Flash Debug/zl_mirror.o
 .bss           0x40001aa4       0x1c ARM Flash Debug/zl_event.o
 .bss           0x40001ac0       0x44 ARM Flash Debug/icmp.o
 .bss           0x40001b04        0x4 ARM Flash Debug/pm.o
 .bss           0x40001b08       0x28 ARM Flash Debug/zl_ctrl1.o
 .bss           0x40001b30       0x28 ARM Flash Debug/zl_ctrl2.o
 .bss           0x40001b58       0x58 ARM Flash Debug/nvstore.o
 .bss           0x40001bb0       0x28 ARM Flash Debug/trunk.o
 .bss           0x40001bd8       0x68 ARM Flash Debug/uip_arp.o
 .bss           0x40001c40       0x1c ARM Flash Debug/fs.o
 .bss           0x40001c5c       0xac ARM Flash Debug/telnetd.o
 .bss           0x40001d08        0xc ARM Flash Debug/uip.o
 *(COMMON)
 COMMON         0x40001d14      0x300 ARM Flash Debug/cli.o
                0x40001d14                handlerTable
 COMMON         0x40002014       0x10 ARM Flash Debug/sfp.o
                0x40002014                modulePresent
 COMMON         0x40002024        0x4 ARM Flash Debug/httpd.o
                0x40002024                hs
 COMMON         0x40002028      0x970 ARM Flash Debug/uip.o
                0x40002028                uip_len
                0x4000202c                uip_sappdata
                0x40002030                uip_acc32
                0x40002034                uip_flags
                0x40002038                uip_appdata
                0x4000203c                uip_conn
                0x40002040                uip_conns
                0x40002360                uip_listenports
                0x40002388                uip_stat
                0x400023b8                uip_buf
                0x40002996                uip_slen
 COMMON         0x40002998        0x4 E:/Program Files/Rowley Associates Limited/CrossWorks for ARM 1.3/lib/libc_v4t_a_ni_le.a(errno.o)
                0x40002998                errno
                0x4000299c                __bss_end__ = (__bss_start__ + SIZEOF (.bss))
                0x00000001                . = ASSERT (((__bss_end__ >= __SRAM_segment_start__) && (__bss_end__ <= (__SRAM_segment_start__ + 0x10000))), .bss is too large to fit in SRAM memory segment)

.heap           0x4000299c      0x400
                0x4000299c                __heap_start__ = .
 *(.heap)
                0x40002d9c                . = ((__heap_start__ + 0x400) MAX_K .)
 *fill*         0x4000299c      0x400 00
                0x40002d9c                __heap_end__ = (__heap_start__ + SIZEOF (.heap))
                0x00000001                . = ASSERT (((__heap_end__ >= __SRAM_segment_start__) && (__heap_end__ <= (__SRAM_segment_start__ + 0x10000))), .heap is too large to fit in SRAM memory segment)

.stack          0x40002d9c      0x400
                0x40002d9c                __stack_start__ = .
 *(.stack)
                0x4000319c                . = ((__stack_start__ + 0x400) MAX_K .)
 *fill*         0x40002d9c      0x400 00
                0x4000319c                __stack_end__ = (__stack_start__ + SIZEOF (.stack))
                0x00000001                . = ASSERT (((__stack_end__ >= __SRAM_segment_start__) && (__stack_end__ <= (__SRAM_segment_start__ + 0x10000))), .stack is too large to fit in SRAM memory segment)

.stack_irq      0x4000319c      0x100
                0x4000319c                __stack_irq_start__ = .
 *(.stack_irq)
                0x4000329c                . = ((__stack_irq_start__ + 0x100) MAX_K .)
 *fill*         0x4000319c      0x100 00
                0x4000329c                __stack_irq_end__ = (__stack_irq_start__ + SIZEOF (.stack_irq))
                0x00000001                . = ASSERT (((__stack_irq_end__ >= __SRAM_segment_start__) && (__stack_irq_end__ <= (__SRAM_segment_start__ + 0x10000))), .stack_irq is too large to fit in SRAM memory segment)

.stack_fiq      0x4000329c      0x100
                0x4000329c                __stack_fiq_start__ = .
 *(.stack_fiq)
                0x4000339c                . = ((__stack_fiq_start__ + 0x100) MAX_K .)
 *fill*         0x4000329c      0x100 00
                0x4000339c                __stack_fiq_end__ = (__stack_fiq_start__ + SIZEOF (.stack_fiq))
                0x00000001                . = ASSERT (((__stack_fiq_end__ >= __SRAM_segment_start__) && (__stack_fiq_end__ <= (__SRAM_segment_start__ + 0x10000))), .stack_fiq is too large to fit in SRAM memory segment)

.stack_svc      0x4000339c        0x0
                0x4000339c                __stack_svc_start__ = .
 *(.stack_svc)
                0x4000339c                . = ((__stack_svc_start__ + 0x0) MAX_K .)
                0x4000339c                __stack_svc_end__ = (__stack_svc_start__ + SIZEOF (.stack_svc))
                0x00000001                . = ASSERT (((__stack_svc_end__ >= __SRAM_segment_start__) && (__stack_svc_end__ <= (__SRAM_segment_start__ + 0x10000))), .stack_svc is too large to fit in SRAM memory segment)

.stack_abt      0x4000339c        0x0
                0x4000339c                __stack_abt_start__ = .
 *(.stack_abt)
                0x4000339c                . = ((__stack_abt_start__ + 0x0) MAX_K .)
                0x4000339c                __stack_abt_end__ = (__stack_abt_start__ + SIZEOF (.stack_abt))
                0x00000001                . = ASSERT (((__stack_abt_end__ >= __SRAM_segment_start__) && (__stack_abt_end__ <= (__SRAM_segment_start__ + 0x10000))), .stack_abt is too large to fit in SRAM memory segment)

.stack_und      0x4000339c        0x0
                0x4000339c                __stack_und_start__ = .
 *(.stack_und)
                0x4000339c                . = ((__stack_und_start__ + 0x0) MAX_K .)
                0x4000339c                __stack_und_end__ = (__stack_und_start__ + SIZEOF (.stack_und))
                0x00000001                . = ASSERT (((__stack_und_end__ >= __SRAM_segment_start__) && (__stack_und_end__ <= (__SRAM_segment_start__ + 0x10000))), .stack_und is too large to fit in SRAM memory segment)
START GROUP
LOAD ARM Flash Debug/zarlink.o
LOAD ARM Flash Debug/armvic.o
LOAD ARM Flash Debug/board.o
LOAD ARM Flash Debug/charconv.o
LOAD ARM Flash Debug/cli.o
LOAD ARM Flash Debug/clichar.o
LOAD ARM Flash Debug/clivar.o
LOAD ARM Flash Debug/crc8.o
LOAD ARM Flash Debug/crc16.o
LOAD ARM Flash Debug/ee24lc256.o
LOAD ARM Flash Debug/eventq.o
LOAD ARM Flash Debug/i2cmaster.o
LOAD ARM Flash Debug/i2cport.o
LOAD ARM Flash Debug/i2cswitch.o
LOAD ARM Flash Debug/init.o
LOAD ARM Flash Debug/medusa.o
LOAD ARM Flash Debug/nohau.o
LOAD ARM Flash Debug/olimex.o
LOAD ARM Flash Debug/pll.o
LOAD ARM Flash Debug/sfpdiag.o
LOAD ARM Flash Debug/spi.o
LOAD ARM Flash Debug/spiprot.o
LOAD ARM Flash Debug/timer0.o
LOAD ARM Flash Debug/uart0.o
LOAD ARM Flash Debug/watchdog.o
LOAD ARM Flash Debug/xmodem.o
LOAD ARM Flash Debug/sfp.o
LOAD ARM Flash Debug/strutil.o
LOAD ARM Flash Debug/zl_ssi.o
LOAD ARM Flash Debug/zl_rmon.o
LOAD ARM Flash Debug/zl_frame.o
LOAD ARM Flash Debug/zl_mii.o
LOAD ARM Flash Debug/zl_bus.o
LOAD ARM Flash Debug/zl_util.o
LOAD ARM Flash Debug/zl_mirror.o
LOAD ARM Flash Debug/zl_event.o
LOAD ARM Flash Debug/icmp.o
LOAD ARM Flash Debug/pm.o
LOAD ARM Flash Debug/armirq.o
LOAD ARM Flash Debug/spimesg.o
LOAD ARM Flash Debug/medusa_rev2.o
LOAD ARM Flash Debug/ssp.o
LOAD ARM Flash Debug/zl_ctrl1.o
LOAD ARM Flash Debug/zl_ctrl2.o
LOAD ARM Flash Debug/zl_reset.o
LOAD ARM Flash Debug/ip.o
LOAD ARM Flash Debug/nvstore.o
LOAD ARM Flash Debug/zl_rxframe.o
LOAD ARM Flash Debug/trunk.o
LOAD ARM Flash Debug/crt0.o
LOAD ARM Flash Debug/Philips_LPC210X_Startup.o
LOAD ARM Flash Debug/uip_arp.o
LOAD ARM Flash Debug/cgi.o
LOAD ARM Flash Debug/fs.o
LOAD ARM Flash Debug/httpd.o
LOAD ARM Flash Debug/memb.o
LOAD ARM Flash Debug/telnetd.o
LOAD ARM Flash Debug/telnetd-shell.o
LOAD ARM Flash Debug/uip.o
LOAD ARM Flash Debug/uip_arch.o
LOAD E:/Program Files/Rowley Associates Limited/CrossWorks for ARM 1.3/lib/libarmdi_v4t_a_ni_le.a
LOAD E:/Program Files/Rowley Associates Limited/CrossWorks for ARM 1.3/lib/libm_v4t_a_ni_le.a
LOAD E:/Program Files/Rowley Associates Limited/CrossWorks for ARM 1.3/lib/libc_v4t_a_ni_le.a
LOAD E:/Program Files/Rowley Associates Limited/CrossWorks for ARM 1.3/lib/libcpp_v4t_a_ni_le.a
LOAD E:/Program Files/Rowley Associates Limited/CrossWorks for ARM 1.3/lib/libm_v4t_a_ni_le.a
LOAD E:/Program Files/Rowley Associates Limited/CrossWorks for ARM 1.3/lib/libc_v4t_a_ni_le.a
LOAD E:/Program Files/Rowley Associates Limited/CrossWorks for ARM 1.3/lib/lib_vfprintf_double_long_long_v4t_a_ni_le.a
LOAD E:/Program Files/Rowley Associates Limited/CrossWorks for ARM 1.3/lib/lib_vfscanf_long_v4t_a_ni_le.a
END GROUP
OUTPUT(ARM Flash Debug/medusa.elf elf32-littlearm)

.debug_abbrev   0x00000000     0x2f81
 .debug_abbrev  0x00000000       0x76 ARM Flash Debug/zarlink.o
 .debug_abbrev  0x00000076       0xc3 ARM Flash Debug/armvic.o
 .debug_abbrev  0x00000139       0xbe ARM Flash Debug/board.o
 .debug_abbrev  0x000001f7       0x1f ARM Flash Debug/charconv.o
 .debug_abbrev  0x00000216      0x123 ARM Flash Debug/cli.o
 .debug_abbrev  0x00000339      0x11f ARM Flash Debug/clichar.o
 .debug_abbrev  0x00000458       0xd7 ARM Flash Debug/clivar.o
 .debug_abbrev  0x0000052f       0x1f ARM Flash Debug/crc8.o
 .debug_abbrev  0x0000054e       0x97 ARM Flash Debug/crc16.o
 .debug_abbrev  0x000005e5      0x121 ARM Flash Debug/ee24lc256.o
 .debug_abbrev  0x00000706       0xbf ARM Flash Debug/eventq.o
 .debug_abbrev  0x000007c5      0x15f ARM Flash Debug/i2cmaster.o
 .debug_abbrev  0x00000924       0xa2 ARM Flash Debug/i2cport.o
 .debug_abbrev  0x000009c6       0x8d ARM Flash Debug/i2cswitch.o
 .debug_abbrev  0x00000a53       0xe6 ARM Flash Debug/init.o
 .debug_abbrev  0x00000b39       0x8d ARM Flash Debug/medusa.o
 .debug_abbrev  0x00000bc6       0x1f ARM Flash Debug/nohau.o
 .debug_abbrev  0x00000be5       0x1f ARM Flash Debug/olimex.o
 .debug_abbrev  0x00000c04       0xa9 ARM Flash Debug/pll.o
 .debug_abbrev  0x00000cad      0x1a6 ARM Flash Debug/sfpdiag.o
 .debug_abbrev  0x00000e53      0x12a ARM Flash Debug/spi.o
 .debug_abbrev  0x00000f7d       0x1f ARM Flash Debug/spiprot.o
 .debug_abbrev  0x00000f9c       0x97 ARM Flash Debug/timer0.o
 .debug_abbrev  0x00001033      0x122 ARM Flash Debug/uart0.o
 .debug_abbrev  0x00001155       0xc5 ARM Flash Debug/watchdog.o
 .debug_abbrev  0x0000121a       0x1f ARM Flash Debug/xmodem.o
 .debug_abbrev  0x00001239       0xe8 ARM Flash Debug/sfp.o
 .debug_abbrev  0x00001321       0x93 ARM Flash Debug/strutil.o
 .debug_abbrev  0x000013b4       0xb4 ARM Flash Debug/zl_ssi.o
 .debug_abbrev  0x00001468      0x1d2 ARM Flash Debug/zl_rmon.o
 .debug_abbrev  0x0000163a      0x124 ARM Flash Debug/zl_frame.o
 .debug_abbrev  0x0000175e       0xe2 ARM Flash Debug/zl_mii.o
 .debug_abbrev  0x00001840      0x11f ARM Flash Debug/zl_bus.o
 .debug_abbrev  0x0000195f      0x1bc ARM Flash Debug/zl_util.o
 .debug_abbrev  0x00001b1b       0xe0 ARM Flash Debug/zl_mirror.o
 .debug_abbrev  0x00001bfb       0xcd ARM Flash Debug/zl_event.o
 .debug_abbrev  0x00001cc8       0xe4 ARM Flash Debug/icmp.o
 .debug_abbrev  0x00001dac       0xae ARM Flash Debug/pm.o
 .debug_abbrev  0x00001e5a       0xa8 ARM Flash Debug/armirq.o
 .debug_abbrev  0x00001f02       0x1f ARM Flash Debug/spimesg.o
 .debug_abbrev  0x00001f21       0x1f ARM Flash Debug/medusa_rev2.o
 .debug_abbrev  0x00001f40       0x1f ARM Flash Debug/ssp.o
 .debug_abbrev  0x00001f5f       0xd7 ARM Flash Debug/zl_ctrl1.o
 .debug_abbrev  0x00002036       0xa6 ARM Flash Debug/zl_ctrl2.o
 .debug_abbrev  0x000020dc       0x63 ARM Flash Debug/zl_reset.o
 .debug_abbrev  0x0000213f       0xaa ARM Flash Debug/ip.o
 .debug_abbrev  0x000021e9      0x16a ARM Flash Debug/nvstore.o
 .debug_abbrev  0x00002353       0x8b ARM Flash Debug/zl_rxframe.o
 .debug_abbrev  0x000023de       0xdc ARM Flash Debug/trunk.o
 .debug_abbrev  0x000024ba       0x14 ARM Flash Debug/crt0.o
 .debug_abbrev  0x000024ce       0x10 ARM Flash Debug/Philips_LPC210X_Startup.o
 .debug_abbrev  0x000024de      0x17b ARM Flash Debug/uip_arp.o
 .debug_abbrev  0x00002659      0x123 ARM Flash Debug/cgi.o
 .debug_abbrev  0x0000277c      0x107 ARM Flash Debug/fs.o
 .debug_abbrev  0x00002883      0x176 ARM Flash Debug/httpd.o
 .debug_abbrev  0x000029f9       0xab ARM Flash Debug/memb.o
 .debug_abbrev  0x00002aa4      0x175 ARM Flash Debug/telnetd.o
 .debug_abbrev  0x00002c19      0x106 ARM Flash Debug/telnetd-shell.o
 .debug_abbrev  0x00002d1f      0x18c ARM Flash Debug/uip.o
 .debug_abbrev  0x00002eab       0xd6 ARM Flash Debug/uip_arch.o

.debug_info     0x00000000     0xd8b3
 .debug_info    0x00000000      0x14b ARM Flash Debug/zarlink.o
 .debug_info    0x0000014b      0x3e6 ARM Flash Debug/armvic.o
 .debug_info    0x00000531      0x2a1 ARM Flash Debug/board.o
 .debug_info    0x000007d2       0x5c ARM Flash Debug/charconv.o
 .debug_info    0x0000082e      0x586 ARM Flash Debug/cli.o
 .debug_info    0x00000db4      0x41f ARM Flash Debug/clichar.o
 .debug_info    0x000011d3      0x274 ARM Flash Debug/clivar.o
 .debug_info    0x00001447       0x58 ARM Flash Debug/crc8.o
 .debug_info    0x0000149f      0x1d4 ARM Flash Debug/crc16.o
 .debug_info    0x00001673      0x6dd ARM Flash Debug/ee24lc256.o
 .debug_info    0x00001d50      0x451 ARM Flash Debug/eventq.o
 .debug_info    0x000021a1      0x862 ARM Flash Debug/i2cmaster.o
 .debug_info    0x00002a03      0x482 ARM Flash Debug/i2cport.o
 .debug_info    0x00002e85      0x20e ARM Flash Debug/i2cswitch.o
 .debug_info    0x00003093      0x3d7 ARM Flash Debug/init.o
 .debug_info    0x0000346a      0x174 ARM Flash Debug/medusa.o
 .debug_info    0x000035de       0x59 ARM Flash Debug/nohau.o
 .debug_info    0x00003637       0x5a ARM Flash Debug/olimex.o
 .debug_info    0x00003691      0x20f ARM Flash Debug/pll.o
 .debug_info    0x000038a0      0x8ec ARM Flash Debug/sfpdiag.o
 .debug_info    0x0000418c      0x5bb ARM Flash Debug/spi.o
 .debug_info    0x00004747       0x63 ARM Flash Debug/spiprot.o
 .debug_info    0x000047aa      0x1c2 ARM Flash Debug/timer0.o
 .debug_info    0x0000496c      0x570 ARM Flash Debug/uart0.o
 .debug_info    0x00004edc      0x19b ARM Flash Debug/watchdog.o
 .debug_info    0x00005077       0x5a ARM Flash Debug/xmodem.o
 .debug_info    0x000050d1      0x351 ARM Flash Debug/sfp.o
 .debug_info    0x00005422      0x1fb ARM Flash Debug/strutil.o
 .debug_info    0x0000561d      0x37e ARM Flash Debug/zl_ssi.o
 .debug_info    0x0000599b      0xc79 ARM Flash Debug/zl_rmon.o
 .debug_info    0x00006614      0x377 ARM Flash Debug/zl_frame.o
 .debug_info    0x0000698b      0x4fd ARM Flash Debug/zl_mii.o
 .debug_info    0x00006e88      0x594 ARM Flash Debug/zl_bus.o
 .debug_info    0x0000741c      0xab2 ARM Flash Debug/zl_util.o
 .debug_info    0x00007ece      0x2f9 ARM Flash Debug/zl_mirror.o
 .debug_info    0x000081c7      0x45a ARM Flash Debug/zl_event.o
 .debug_info    0x00008621      0x47e ARM Flash Debug/icmp.o
 .debug_info    0x00008a9f      0x19b ARM Flash Debug/pm.o
 .debug_info    0x00008c3a      0x23b ARM Flash Debug/armirq.o
 .debug_info    0x00008e75       0x63 ARM Flash Debug/spimesg.o
 .debug_info    0x00008ed8       0x5f ARM Flash Debug/medusa_rev2.o
 .debug_info    0x00008f37       0x91 ARM Flash Debug/ssp.o
 .debug_info    0x00008fc8      0x2b4 ARM Flash Debug/zl_ctrl1.o
 .debug_info    0x0000927c      0x17d ARM Flash Debug/zl_ctrl2.o
 .debug_info    0x000093f9      0x107 ARM Flash Debug/zl_reset.o
 .debug_info    0x00009500      0x1be ARM Flash Debug/ip.o
 .debug_info    0x000096be      0x976 ARM Flash Debug/nvstore.o
 .debug_info    0x0000a034      0x152 ARM Flash Debug/zl_rxframe.o
 .debug_info    0x0000a186      0x31c ARM Flash Debug/trunk.o
 .debug_info    0x0000a4a2       0x8d ARM Flash Debug/crt0.o
 .debug_info    0x0000a52f       0xa9 ARM Flash Debug/Philips_LPC210X_Startup.o
 .debug_info    0x0000a5d8      0x3bd ARM Flash Debug/uip_arp.o
 .debug_info    0x0000a995      0x7d8 ARM Flash Debug/cgi.o
 .debug_info    0x0000b16d      0x90c ARM Flash Debug/fs.o
 .debug_info    0x0000ba79      0x4cd ARM Flash Debug/httpd.o
 .debug_info    0x0000bf46      0x1dc ARM Flash Debug/memb.o
 .debug_info    0x0000c122      0x679 ARM Flash Debug/telnetd.o
 .debug_info    0x0000c79b      0x59b ARM Flash Debug/telnetd-shell.o
 .debug_info    0x0000cd36      0x94a ARM Flash Debug/uip.o
 .debug_info    0x0000d680      0x233 ARM Flash Debug/uip_arch.o

.debug_line     0x00000000     0x25db
 .debug_line    0x00000000       0x6a ARM Flash Debug/zarlink.o
 .debug_line    0x0000006a       0x8c ARM Flash Debug/armvic.o
 .debug_line    0x000000f6       0x79 ARM Flash Debug/board.o
 .debug_line    0x0000016f       0x1a ARM Flash Debug/charconv.o
 .debug_line    0x00000189       0xc1 ARM Flash Debug/cli.o
 .debug_line    0x0000024a       0xb4 ARM Flash Debug/clichar.o
 .debug_line    0x000002fe       0x50 ARM Flash Debug/clivar.o
 .debug_line    0x0000034e       0x1a ARM Flash Debug/crc8.o
 .debug_line    0x00000368       0x55 ARM Flash Debug/crc16.o
 .debug_line    0x000003bd       0xe3 ARM Flash Debug/ee24lc256.o
 .debug_line    0x000004a0       0x9a ARM Flash Debug/eventq.o
 .debug_line    0x0000053a      0x151 ARM Flash Debug/i2cmaster.o
 .debug_line    0x0000068b       0x8e ARM Flash Debug/i2cport.o
 .debug_line    0x00000719       0x63 ARM Flash Debug/i2cswitch.o
 .debug_line    0x0000077c       0xa8 ARM Flash Debug/init.o
 .debug_line    0x00000824       0x62 ARM Flash Debug/medusa.o
 .debug_line    0x00000886       0x1a ARM Flash Debug/nohau.o
 .debug_line    0x000008a0       0x1a ARM Flash Debug/olimex.o
 .debug_line    0x000008ba       0x73 ARM Flash Debug/pll.o
 .debug_line    0x0000092d      0x115 ARM Flash Debug/sfpdiag.o
 .debug_line    0x00000a42       0xb2 ARM Flash Debug/spi.o
 .debug_line    0x00000af4       0x1a ARM Flash Debug/spiprot.o
 .debug_line    0x00000b0e       0x6d ARM Flash Debug/timer0.o
 .debug_line    0x00000b7b       0xd2 ARM Flash Debug/uart0.o
 .debug_line    0x00000c4d       0x5d ARM Flash Debug/watchdog.o
 .debug_line    0x00000caa       0x1a ARM Flash Debug/xmodem.o
 .debug_line    0x00000cc4       0xa1 ARM Flash Debug/sfp.o
 .debug_line    0x00000d65       0x67 ARM Flash Debug/strutil.o
 .debug_line    0x00000dcc       0xb8 ARM Flash Debug/zl_ssi.o
 .debug_line    0x00000e84      0x25d ARM Flash Debug/zl_rmon.o
 .debug_line    0x000010e1      0x123 ARM Flash Debug/zl_frame.o
 .debug_line    0x00001204       0xe4 ARM Flash Debug/zl_mii.o
 .debug_line    0x000012e8       0xd1 ARM Flash Debug/zl_bus.o
 .debug_line    0x000013b9      0x164 ARM Flash Debug/zl_util.o
 .debug_line    0x0000151d       0x9c ARM Flash Debug/zl_mirror.o
 .debug_line    0x000015b9       0xb1 ARM Flash Debug/zl_event.o
 .debug_line    0x0000166a       0x99 ARM Flash Debug/icmp.o
 .debug_line    0x00001703       0x51 ARM Flash Debug/pm.o
 .debug_line    0x00001754       0x69 ARM Flash Debug/armirq.o
 .debug_line    0x000017bd       0x1a ARM Flash Debug/spimesg.o
 .debug_line    0x000017d7       0x1a ARM Flash Debug/medusa_rev2.o
 .debug_line    0x000017f1       0x1a ARM Flash Debug/ssp.o
 .debug_line    0x0000180b       0x72 ARM Flash Debug/zl_ctrl1.o
 .debug_line    0x0000187d       0x50 ARM Flash Debug/zl_ctrl2.o
 .debug_line    0x000018cd       0x49 ARM Flash Debug/zl_reset.o
 .debug_line    0x00001916       0x51 ARM Flash Debug/ip.o
 .debug_line    0x00001967      0x165 ARM Flash Debug/nvstore.o
 .debug_line    0x00001acc       0x7a ARM Flash Debug/zl_rxframe.o
 .debug_line    0x00001b46       0x5b ARM Flash Debug/trunk.o
 .debug_line    0x00001ba1       0xe6 ARM Flash Debug/crt0.o
 .debug_line    0x00001c87       0xc8 ARM Flash Debug/Philips_LPC210X_Startup.o
 .debug_line    0x00001d4f       0xf2 ARM Flash Debug/uip_arp.o
 .debug_line    0x00001e41       0x98 ARM Flash Debug/cgi.o
 .debug_line    0x00001ed9       0x9a ARM Flash Debug/fs.o
 .debug_line    0x00001f73       0xed ARM Flash Debug/httpd.o
 .debug_line    0x00002060       0x73 ARM Flash Debug/memb.o
 .debug_line    0x000020d3      0x10d ARM Flash Debug/telnetd.o
 .debug_line    0x000021e0       0xba ARM Flash Debug/telnetd-shell.o
 .debug_line    0x0000229a      0x29f ARM Flash Debug/uip.o
 .debug_line    0x00002539       0xa2 ARM Flash Debug/uip_arch.o

.debug_frame    0x00000000     0x3f9c
 .debug_frame   0x00000000       0x3c ARM Flash Debug/zarlink.o
 .debug_frame   0x0000003c      0x224 ARM Flash Debug/armvic.o
 .debug_frame   0x00000260      0x19c ARM Flash Debug/board.o
 .debug_frame   0x000003fc      0x19c ARM Flash Debug/cli.o
 .debug_frame   0x00000598      0x220 ARM Flash Debug/clichar.o
 .debug_frame   0x000007b8       0x68 ARM Flash Debug/clivar.o
 .debug_frame   0x00000820       0xc0 ARM Flash Debug/crc16.o
 .debug_frame   0x000008e0      0x24c ARM Flash Debug/ee24lc256.o
 .debug_frame   0x00000b2c      0x144 ARM Flash Debug/eventq.o
 .debug_frame   0x00000c70      0x304 ARM Flash Debug/i2cmaster.o
 .debug_frame   0x00000f74      0x19c ARM Flash Debug/i2cport.o
 .debug_frame   0x00001110       0xc0 ARM Flash Debug/i2cswitch.o
 .debug_frame   0x000011d0       0x3c ARM Flash Debug/init.o
 .debug_frame   0x0000120c       0xec ARM Flash Debug/medusa.o
 .debug_frame   0x000012f8      0x144 ARM Flash Debug/pll.o
 .debug_frame   0x0000143c      0x280 ARM Flash Debug/sfpdiag.o
 .debug_frame   0x000016bc      0x14c ARM Flash Debug/spi.o
 .debug_frame   0x00001808       0xc8 ARM Flash Debug/timer0.o
 .debug_frame   0x000018d0      0x1a4 ARM Flash Debug/uart0.o
 .debug_frame   0x00001a74      0x118 ARM Flash Debug/watchdog.o
 .debug_frame   0x00001b8c      0x118 ARM Flash Debug/sfp.o
 .debug_frame   0x00001ca4       0x68 ARM Flash Debug/strutil.o
 .debug_frame   0x00001d0c      0x24c ARM Flash Debug/zl_ssi.o
 .debug_frame   0x00001f58      0x278 ARM Flash Debug/zl_rmon.o
 .debug_frame   0x000021d0       0x68 ARM Flash Debug/zl_frame.o
 .debug_frame   0x00002238      0x170 ARM Flash Debug/zl_mii.o
 .debug_frame   0x000023a8      0x3d8 ARM Flash Debug/zl_bus.o
 .debug_frame   0x00002780      0x2a4 ARM Flash Debug/zl_util.o
 .debug_frame   0x00002a24       0xec ARM Flash Debug/zl_mirror.o
 .debug_frame   0x00002b10      0x178 ARM Flash Debug/zl_event.o
 .debug_frame   0x00002c88      0x144 ARM Flash Debug/icmp.o
 .debug_frame   0x00002dcc       0xc0 ARM Flash Debug/pm.o
 .debug_frame   0x00002e8c      0x170 ARM Flash Debug/armirq.o
 .debug_frame   0x00002ffc       0xc0 ARM Flash Debug/zl_ctrl1.o
 .debug_frame   0x000030bc       0x94 ARM Flash Debug/zl_ctrl2.o
 .debug_frame   0x00003150       0x68 ARM Flash Debug/zl_reset.o
 .debug_frame   0x000031b8       0x94 ARM Flash Debug/ip.o
 .debug_frame   0x0000324c      0x220 ARM Flash Debug/nvstore.o
 .debug_frame   0x0000346c       0x68 ARM Flash Debug/zl_rxframe.o
 .debug_frame   0x000034d4      0x118 ARM Flash Debug/trunk.o
 .debug_frame   0x000035ec      0x118 ARM Flash Debug/uip_arp.o
 .debug_frame   0x00003704       0x98 ARM Flash Debug/cgi.o
 .debug_frame   0x0000379c       0xc0 ARM Flash Debug/fs.o
 .debug_frame   0x0000385c       0xc0 ARM Flash Debug/httpd.o
 .debug_frame   0x0000391c       0xc0 ARM Flash Debug/memb.o
 .debug_frame   0x000039dc      0x24c ARM Flash Debug/telnetd.o
 .debug_frame   0x00003c28      0x170 ARM Flash Debug/telnetd-shell.o
 .debug_frame   0x00003d98      0x144 ARM Flash Debug/uip.o
 .debug_frame   0x00003edc       0xc0 ARM Flash Debug/uip_arch.o

.debug_pubnames
                0x00000000     0x1480
 .debug_pubnames
                0x00000000       0x22 ARM Flash Debug/zarlink.o
 .debug_pubnames
                0x00000022       0xec ARM Flash Debug/armvic.o
 .debug_pubnames
                0x0000010e       0x70 ARM Flash Debug/board.o
 .debug_pubnames
                0x0000017e       0x67 ARM Flash Debug/cli.o
 .debug_pubnames
                0x000001e5       0x91 ARM Flash Debug/clichar.o
 .debug_pubnames
                0x00000276       0x38 ARM Flash Debug/clivar.o
 .debug_pubnames
                0x000002ae       0x51 ARM Flash Debug/crc16.o
 .debug_pubnames
                0x000002ff       0xae ARM Flash Debug/ee24lc256.o
 .debug_pubnames
                0x000003ad       0x93 ARM Flash Debug/eventq.o
 .debug_pubnames
                0x00000440       0xc0 ARM Flash Debug/i2cmaster.o
 .debug_pubnames
                0x00000500       0x78 ARM Flash Debug/i2cport.o
 .debug_pubnames
                0x00000578       0x4d ARM Flash Debug/i2cswitch.o
 .debug_pubnames
                0x000005c5       0x2a ARM Flash Debug/init.o
 .debug_pubnames
                0x000005ef       0x81 ARM Flash Debug/medusa.o
 .debug_pubnames
                0x00000670       0x75 ARM Flash Debug/pll.o
 .debug_pubnames
                0x000006e5       0xb7 ARM Flash Debug/sfpdiag.o
 .debug_pubnames
                0x0000079c       0x34 ARM Flash Debug/spi.o
 .debug_pubnames
                0x000007d0       0x44 ARM Flash Debug/timer0.o
 .debug_pubnames
                0x00000814       0x69 ARM Flash Debug/uart0.o
 .debug_pubnames
                0x0000087d       0x34 ARM Flash Debug/watchdog.o
 .debug_pubnames
                0x000008b1       0x77 ARM Flash Debug/sfp.o
 .debug_pubnames
                0x00000928       0x3d ARM Flash Debug/strutil.o
 .debug_pubnames
                0x00000965       0x73 ARM Flash Debug/zl_rmon.o
 .debug_pubnames
                0x000009d8       0x56 ARM Flash Debug/zl_frame.o
 .debug_pubnames
                0x00000a2e       0x94 ARM Flash Debug/zl_mii.o
 .debug_pubnames
                0x00000ac2      0x14c ARM Flash Debug/zl_bus.o
 .debug_pubnames
                0x00000c0e       0xa5 ARM Flash Debug/zl_util.o
 .debug_pubnames
                0x00000cb3       0x28 ARM Flash Debug/zl_mirror.o
 .debug_pubnames
                0x00000cdb       0x73 ARM Flash Debug/zl_event.o
 .debug_pubnames
                0x00000d4e       0x4b ARM Flash Debug/icmp.o
 .debug_pubnames
                0x00000d99       0x34 ARM Flash Debug/pm.o
 .debug_pubnames
                0x00000dcd       0x6a ARM Flash Debug/armirq.o
 .debug_pubnames
                0x00000e37       0x44 ARM Flash Debug/zl_ctrl1.o
 .debug_pubnames
                0x00000e7b       0x44 ARM Flash Debug/zl_ctrl2.o
 .debug_pubnames
                0x00000ebf       0x27 ARM Flash Debug/zl_reset.o
 .debug_pubnames
                0x00000ee6       0x2b ARM Flash Debug/ip.o
 .debug_pubnames
                0x00000f11       0x43 ARM Flash Debug/nvstore.o
 .debug_pubnames
                0x00000f54       0x29 ARM Flash Debug/zl_rxframe.o
 .debug_pubnames
                0x00000f7d       0x41 ARM Flash Debug/trunk.o
 .debug_pubnames
                0x00000fbe       0x78 ARM Flash Debug/uip_arp.o
 .debug_pubnames
                0x00001036       0x1d ARM Flash Debug/cgi.o
 .debug_pubnames
                0x00001053      0x173 ARM Flash Debug/fs.o
 .debug_pubnames
                0x000011c6       0x3a ARM Flash Debug/httpd.o
 .debug_pubnames
                0x00001200       0x4a ARM Flash Debug/memb.o
 .debug_pubnames
                0x0000124a       0x6b ARM Flash Debug/telnetd.o
 .debug_pubnames
                0x000012b5       0x3a ARM Flash Debug/telnetd-shell.o
 .debug_pubnames
                0x000012ef      0x13f ARM Flash Debug/uip.o
 .debug_pubnames
                0x0000142e       0x52 ARM Flash Debug/uip_arch.o

.debug_aranges  0x00000000      0x668
 .debug_aranges
                0x00000000       0x20 ARM Flash Debug/zarlink.o
 .debug_aranges
                0x00000020       0x20 ARM Flash Debug/armvic.o
 .debug_aranges
                0x00000040       0x20 ARM Flash Debug/board.o
 .debug_aranges
                0x00000060       0x20 ARM Flash Debug/cli.o
 .debug_aranges
                0x00000080       0x20 ARM Flash Debug/clichar.o
 .debug_aranges
                0x000000a0       0x20 ARM Flash Debug/clivar.o
 .debug_aranges
                0x000000c0       0x20 ARM Flash Debug/crc16.o
 .debug_aranges
                0x000000e0       0x20 ARM Flash Debug/ee24lc256.o
 .debug_aranges
                0x00000100       0x20 ARM Flash Debug/eventq.o
 .debug_aranges
                0x00000120       0x20 ARM Flash Debug/i2cmaster.o
 .debug_aranges
                0x00000140       0x20 ARM Flash Debug/i2cport.o
 .debug_aranges
                0x00000160       0x20 ARM Flash Debug/i2cswitch.o
 .debug_aranges
                0x00000180       0x20 ARM Flash Debug/init.o
 .debug_aranges
                0x000001a0       0x20 ARM Flash Debug/medusa.o
 .debug_aranges
                0x000001c0       0x20 ARM Flash Debug/pll.o
 .debug_aranges
                0x000001e0       0x20 ARM Flash Debug/sfpdiag.o
 .debug_aranges
                0x00000200       0x20 ARM Flash Debug/spi.o
 .debug_aranges
                0x00000220       0x20 ARM Flash Debug/timer0.o
 .debug_aranges
                0x00000240       0x20 ARM Flash Debug/uart0.o
 .debug_aranges
                0x00000260       0x20 ARM Flash Debug/watchdog.o
 .debug_aranges
                0x00000280       0x20 ARM Flash Debug/sfp.o
 .debug_aranges
                0x000002a0       0x20 ARM Flash Debug/strutil.o
 .debug_aranges
                0x000002c0       0x20 ARM Flash Debug/zl_ssi.o
 .debug_aranges
                0x000002e0       0x20 ARM Flash Debug/zl_rmon.o
 .debug_aranges
                0x00000300       0x20 ARM Flash Debug/zl_frame.o
 .debug_aranges
                0x00000320       0x20 ARM Flash Debug/zl_mii.o
 .debug_aranges
                0x00000340       0x20 ARM Flash Debug/zl_bus.o
 .debug_aranges
                0x00000360       0x20 ARM Flash Debug/zl_util.o
 .debug_aranges
                0x00000380       0x20 ARM Flash Debug/zl_mirror.o
 .debug_aranges
                0x000003a0       0x20 ARM Flash Debug/zl_event.o
 .debug_aranges
                0x000003c0       0x20 ARM Flash Debug/icmp.o
 .debug_aranges
                0x000003e0       0x20 ARM Flash Debug/pm.o
 .debug_aranges
                0x00000400       0x20 ARM Flash Debug/armirq.o
 .debug_aranges
                0x00000420       0x20 ARM Flash Debug/zl_ctrl1.o
 .debug_aranges
                0x00000440       0x20 ARM Flash Debug/zl_ctrl2.o
 .debug_aranges
                0x00000460       0x20 ARM Flash Debug/zl_reset.o
 .debug_aranges
                0x00000480       0x20 ARM Flash Debug/ip.o
 .debug_aranges
                0x000004a0       0x20 ARM Flash Debug/nvstore.o
 .debug_aranges
                0x000004c0       0x20 ARM Flash Debug/zl_rxframe.o
 .debug_aranges
                0x000004e0       0x20 ARM Flash Debug/trunk.o
 .debug_aranges
                0x00000500       0x20 ARM Flash Debug/crt0.o
 .debug_aranges
                0x00000520       0x28 ARM Flash Debug/Philips_LPC210X_Startup.o
 .debug_aranges
                0x00000548       0x20 ARM Flash Debug/uip_arp.o
 .debug_aranges
                0x00000568       0x20 ARM Flash Debug/cgi.o
 .debug_aranges
                0x00000588       0x20 ARM Flash Debug/fs.o
 .debug_aranges
                0x000005a8       0x20 ARM Flash Debug/httpd.o
 .debug_aranges
                0x000005c8       0x20 ARM Flash Debug/memb.o
 .debug_aranges
                0x000005e8       0x20 ARM Flash Debug/telnetd.o
 .debug_aranges
                0x00000608       0x20 ARM Flash Debug/telnetd-shell.o
 .debug_aranges
                0x00000628       0x20 ARM Flash Debug/uip.o
 .debug_aranges
                0x00000648       0x20 ARM Flash Debug/uip_arch.o

.comment        0x00000000      0xbf4
 .comment       0x00000000       0x22 ARM Flash Debug/zarlink.o
 .comment       0x00000022       0x22 ARM Flash Debug/armvic.o
 .comment       0x00000044       0x22 ARM Flash Debug/board.o
 .comment       0x00000066       0x22 ARM Flash Debug/charconv.o
 .comment       0x00000088       0x22 ARM Flash Debug/cli.o
 .comment       0x000000aa       0x22 ARM Flash Debug/clichar.o
 .comment       0x000000cc       0x22 ARM Flash Debug/clivar.o
 .comment       0x000000ee       0x22 ARM Flash Debug/crc8.o
 .comment       0x00000110       0x22 ARM Flash Debug/crc16.o
 .comment       0x00000132       0x22 ARM Flash Debug/ee24lc256.o
 .comment       0x00000154       0x22 ARM Flash Debug/eventq.o
 .comment       0x00000176       0x22 ARM Flash Debug/i2cmaster.o
 .comment       0x00000198       0x22 ARM Flash Debug/i2cport.o
 .comment       0x000001ba       0x22 ARM Flash Debug/i2cswitch.o
 .comment       0x000001dc       0x22 ARM Flash Debug/init.o
 .comment       0x000001fe       0x22 ARM Flash Debug/medusa.o
 .comment       0x00000220       0x22 ARM Flash Debug/nohau.o
 .comment       0x00000242       0x22 ARM Flash Debug/olimex.o
 .comment       0x00000264       0x22 ARM Flash Debug/pll.o
 .comment       0x00000286       0x22 ARM Flash Debug/sfpdiag.o
 .comment       0x000002a8       0x22 ARM Flash Debug/spi.o
 .comment       0x000002ca       0x22 ARM Flash Debug/spiprot.o
 .comment       0x000002ec       0x22 ARM Flash Debug/timer0.o
 .comment       0x0000030e       0x22 ARM Flash Debug/uart0.o
 .comment       0x00000330       0x22 ARM Flash Debug/watchdog.o
 .comment       0x00000352       0x22 ARM Flash Debug/xmodem.o
 .comment       0x00000374       0x22 ARM Flash Debug/sfp.o
 .comment       0x00000396       0x22 ARM Flash Debug/strutil.o
 .comment       0x000003b8       0x22 ARM Flash Debug/zl_ssi.o
 .comment       0x000003da       0x22 ARM Flash Debug/zl_rmon.o
 .comment       0x000003fc       0x22 ARM Flash Debug/zl_frame.o
 .comment       0x0000041e       0x22 ARM Flash Debug/zl_mii.o
 .comment       0x00000440       0x22 ARM Flash Debug/zl_bus.o
 .comment       0x00000462       0x22 ARM Flash Debug/zl_util.o
 .comment       0x00000484       0x22 ARM Flash Debug/zl_mirror.o
 .comment       0x000004a6       0x22 ARM Flash Debug/zl_event.o
 .comment       0x000004c8       0x22 ARM Flash Debug/icmp.o
 .comment       0x000004ea       0x22 ARM Flash Debug/pm.o
 .comment       0x0000050c       0x22 ARM Flash Debug/armirq.o
 .comment       0x0000052e       0x22 ARM Flash Debug/spimesg.o
 .comment       0x00000550       0x22 ARM Flash Debug/medusa_rev2.o
 .comment       0x00000572       0x22 ARM Flash Debug/ssp.o
 .comment       0x00000594       0x22 ARM Flash Debug/zl_ctrl1.o
 .comment       0x000005b6       0x22 ARM Flash Debug/zl_ctrl2.o
 .comment       0x000005d8       0x22 ARM Flash Debug/zl_reset.o
 .comment       0x000005fa       0x22 ARM Flash Debug/ip.o
 .comment       0x0000061c       0x22 ARM Flash Debug/nvstore.o
 .comment       0x0000063e       0x22 ARM Flash Debug/zl_rxframe.o
 .comment       0x00000660       0x22 ARM Flash Debug/trunk.o
 .comment       0x00000682       0x22 ARM Flash Debug/uip_arp.o
 .comment       0x000006a4       0x22 ARM Flash Debug/cgi.o
 .comment       0x000006c6       0x22 ARM Flash Debug/fs.o
 .comment       0x000006e8       0x22 ARM Flash Debug/httpd.o
 .comment       0x0000070a       0x22 ARM Flash Debug/memb.o
 .comment       0x0000072c       0x22 ARM Flash Debug/telnetd.o
 .comment       0x0000074e       0x22 ARM Flash Debug/telnetd-shell.o
 .comment       0x00000770       0x22 ARM Flash Debug/uip.o
 .comment       0x00000792       0x22 ARM Flash Debug/uip_arch.o
 .comment       0x000007b4       0x22 E:/Program Files/Rowley Associates Limited/CrossWorks for ARM 1.3/lib/libc_v4t_a_ni_le.a(strncpy.o)
 .comment       0x000007d6       0x22 E:/Program Files/Rowley Associates Limited/CrossWorks for ARM 1.3/lib/libc_v4t_a_ni_le.a(strtol.o)
 .comment       0x000007f8       0x22 E:/Program Files/Rowley Associates Limited/CrossWorks for ARM 1.3/lib/libc_v4t_a_ni_le.a(errno.o)
 .comment       0x0000081a       0x22 E:/Program Files/Rowley Associates Limited/CrossWorks for ARM 1.3/lib/libc_v4t_a_ni_le.a(printf.o)
 .comment       0x0000083c       0x22 E:/Program Files/Rowley Associates Limited/CrossWorks for ARM 1.3/lib/libc_v4t_a_ni_le.a(sprintf.o)
 .comment       0x0000085e       0x22 E:/Program Files/Rowley Associates Limited/CrossWorks for ARM 1.3/lib/libc_v4t_a_ni_le.a(atoi.o)
 .comment       0x00000880       0x22 E:/Program Files/Rowley Associates Limited/CrossWorks for ARM 1.3/lib/libc_v4t_a_ni_le.a(ctype.o)
 .comment       0x000008a2       0x22 E:/Program Files/Rowley Associates Limited/CrossWorks for ARM 1.3/lib/libc_v4t_a_ni_le.a(__strtoul.o)
 .comment       0x000008c4       0x22 E:/Program Files/Rowley Associates Limited/CrossWorks for ARM 1.3/lib/libc_v4t_a_ni_le.a(__digit.o)
 .comment       0x000008e6       0x22 E:/Program Files/Rowley Associates Limited/CrossWorks for ARM 1.3/lib/lib_vfprintf_double_long_long_v4t_a_ni_le.a(__vfprintf_double_long_long.o)
 .comment       0x00000908       0x22 E:/Program Files/Rowley Associates Limited/CrossWorks for ARM 1.3/lib/libm_v4t_a_ni_le.a(__int64_to_float64.o)
 .comment       0x0000092a       0x22 E:/Program Files/Rowley Associates Limited/CrossWorks for ARM 1.3/lib/libm_v4t_a_ni_le.a(__float32_to_int32.o)
 .comment       0x0000094c       0x22 E:/Program Files/Rowley Associates Limited/CrossWorks for ARM 1.3/lib/libm_v4t_a_ni_le.a(__float32_to_int64.o)
 .comment       0x0000096e       0x22 E:/Program Files/Rowley Associates Limited/CrossWorks for ARM 1.3/lib/libm_v4t_a_ni_le.a(__float32_to_uint32.o)
 .comment       0x00000990       0x22 E:/Program Files/Rowley Associates Limited/CrossWorks for ARM 1.3/lib/libm_v4t_a_ni_le.a(__float32_to_uint64.o)
 .comment       0x000009b2       0x22 E:/Program Files/Rowley Associates Limited/CrossWorks for ARM 1.3/lib/libm_v4t_a_ni_le.a(__float32_to_float64.o)
 .comment       0x000009d4       0x22 E:/Program Files/Rowley Associates Limited/CrossWorks for ARM 1.3/lib/libm_v4t_a_ni_le.a(__float64_to_int32.o)
 .comment       0x000009f6       0x22 E:/Program Files/Rowley Associates Limited/CrossWorks for ARM 1.3/lib/libm_v4t_a_ni_le.a(__float64_to_int64.o)
 .comment       0x00000a18       0x22 E:/Program Files/Rowley Associates Limited/CrossWorks for ARM 1.3/lib/libm_v4t_a_ni_le.a(__float64_to_uint32.o)
 .comment       0x00000a3a       0x22 E:/Program Files/Rowley Associates Limited/CrossWorks for ARM 1.3/lib/libm_v4t_a_ni_le.a(__float64_to_uint64.o)
 .comment       0x00000a5c       0x22 E:/Program Files/Rowley Associates Limited/CrossWorks for ARM 1.3/lib/libm_v4t_a_ni_le.a(__float64_to_float32.o)
 .comment       0x00000a7e       0x22 E:/Program Files/Rowley Associates Limited/CrossWorks for ARM 1.3/lib/libm_v4t_a_ni_le.a(frexp.o)
 .comment       0x00000aa0       0x22 E:/Program Files/Rowley Associates Limited/CrossWorks for ARM 1.3/lib/libm_v4t_a_ni_le.a(ldexp.o)
 .comment       0x00000ac2       0x22 E:/Program Files/Rowley Associates Limited/CrossWorks for ARM 1.3/lib/libm_v4t_a_ni_le.a(__isinf.o)
 .comment       0x00000ae4       0x22 E:/Program Files/Rowley Associates Limited/CrossWorks for ARM 1.3/lib/libm_v4t_a_ni_le.a(__float64_infinity.o)
 .comment       0x00000b06       0x22 E:/Program Files/Rowley Associates Limited/CrossWorks for ARM 1.3/lib/libm_v4t_a_ni_le.a(__isnan.o)
 .comment       0x00000b28       0x22 E:/Program Files/Rowley Associates Limited/CrossWorks for ARM 1.3/lib/libm_v4t_a_ni_le.a(__int32_to_float32.o)
 .comment       0x00000b4a       0x22 E:/Program Files/Rowley Associates Limited/CrossWorks for ARM 1.3/lib/libm_v4t_a_ni_le.a(__int32_to_float64.o)
 .comment       0x00000b6c       0x22 E:/Program Files/Rowley Associates Limited/CrossWorks for ARM 1.3/lib/libm_v4t_a_ni_le.a(__int64_to_float32.o)
 .comment       0x00000b8e       0x22 E:/Program Files/Rowley Associates Limited/CrossWorks for ARM 1.3/lib/libc_v4t_a_ni_le.a(abs.o)
 .comment       0x00000bb0       0x22 E:/Program Files/Rowley Associates Limited/CrossWorks for ARM 1.3/lib/libc_v4t_a_ni_le.a(__pow10.o)
 .comment       0x00000bd2       0x22 E:/Program Files/Rowley Associates Limited/CrossWorks for ARM 1.3/lib/libc_v4t_a_ni_le.a(__hex_lc_uc.o)

.debug_str      0x00000000      0x75e
 .debug_str     0x00000000        0xf ARM Flash Debug/armvic.o
 .debug_str     0x0000000f       0x33 ARM Flash Debug/cli.o
 .debug_str     0x00000042       0x19 ARM Flash Debug/clichar.o
 .debug_str     0x0000005b       0x12 ARM Flash Debug/clivar.o
 .debug_str     0x0000006d       0x13 ARM Flash Debug/crc16.o
 .debug_str     0x00000080       0x62 ARM Flash Debug/ee24lc256.o
 .debug_str     0x000000e2        0x6 ARM Flash Debug/eventq.o
 .debug_str     0x000000e8       0x50 ARM Flash Debug/i2cmaster.o
 .debug_str     0x00000138       0x23 ARM Flash Debug/i2cport.o
 .debug_str     0x0000015b       0x1b ARM Flash Debug/init.o
 .debug_str     0x00000176       0x68 ARM Flash Debug/sfpdiag.o
 .debug_str     0x000001de       0x18 ARM Flash Debug/spi.o
 .debug_str     0x000001f6       0x28 ARM Flash Debug/uart0.o
 .debug_str     0x0000021e       0x23 ARM Flash Debug/sfp.o
 .debug_str     0x00000241       0x12 ARM Flash Debug/strutil.o
 .debug_str     0x00000253        0x9 ARM Flash Debug/zl_ssi.o
 .debug_str     0x0000025c      0x21b ARM Flash Debug/zl_rmon.o
 .debug_str     0x00000477       0x25 ARM Flash Debug/zl_frame.o
 .debug_str     0x0000049c       0x3a ARM Flash Debug/zl_mii.o
 .debug_str     0x000004d6       0x30 ARM Flash Debug/zl_bus.o
 .debug_str     0x00000506       0x4c ARM Flash Debug/zl_util.o
 .debug_str     0x00000552       0x2c ARM Flash Debug/zl_mirror.o
 .debug_str     0x0000057e       0x17 ARM Flash Debug/zl_event.o
 .debug_str     0x00000595       0x28 ARM Flash Debug/icmp.o
 .debug_str     0x000005bd        0x5 ARM Flash Debug/armirq.o
 .debug_str     0x000005c2       0x12 ARM Flash Debug/zl_ctrl1.o
 .debug_str     0x000005d4       0x12 ARM Flash Debug/zl_ctrl2.o
 .debug_str     0x000005e6       0x12 ARM Flash Debug/ip.o
 .debug_str     0x000005f8       0xad ARM Flash Debug/nvstore.o
 .debug_str     0x000006a5       0x12 ARM Flash Debug/zl_rxframe.o
 .debug_str     0x000006b7       0x24 ARM Flash Debug/trunk.o
 .debug_str     0x000006db       0x20 ARM Flash Debug/uip_arp.o
 .debug_str     0x000006fb       0x12 ARM Flash Debug/cgi.o
 .debug_str     0x0000070d       0x1b ARM Flash Debug/httpd.o
 .debug_str     0x00000728       0x1b ARM Flash Debug/telnetd.o
 .debug_str     0x00000743       0x12 ARM Flash Debug/telnetd-shell.o
 .debug_str     0x00000755        0x9 ARM Flash Debug/uip.o
